:100000000C9491010C94A3010C94A3010C949C20DA
:100010000C947A1D0C94A3010C94A3010C94A301DD
:100020000C94A3010C94A3010C94A3010C942A1525
:100030000C94A3010C94A3010C94A3010C94A301B0
:100040000C94DE140C94A3010C941D350C944D32C9
:100050000C94A3010C94A3010C94A3010C94A30190
:100060000C94A3010C94A30109060F0612061506B1
:100070001A0622062A06C506C506C50637063A062A
:1000800043064C06C506C506C506C506C506C50613
:10009000580662066E067606790682068B0691067B
:1000A000C506C5069A06A306AE06E00882148214A9
:1000B000EA08F708040911098214150982142309B2
:1000C00082142D09370941098214821482145109BE
:1000D0005E096B09533555358E358E358E358E3527
:1000E0008E358E358E358E358E358E355B355D355C
:1000F0005F35613563356535673569358E356D3505
:100100006F3571357335753577358E357935084AE4
:10011000D73B3BCE016E84BCBFFDC12F3D6C74311B
:100120009ABD56833DDA3D00C77F11BED9E4BB4C72
:100130003E916BAAAABE000000803F05A84CCDB23C
:10014000D44EB93836A9020C50B9918688083CA61D
:10015000AAAA2ABE000000803F000D0A4772626C06
:1001600020312E3166205B27242720666F7220689D
:10017000656C705D0D0A00244E005B4F50543A00D0
:100180005B5645523A312E31662E32303137303897
:1001900030313A005B544C4F3A005B4739323A00F9
:1001A0003330003238005B4700204700204D0020EC
:1001B000530020460020540033382E005B47433A5A
:1001C00047005B484C503A24242024232024472015
:1001D000244920244E2024783D76616C20244E78DA
:1001E0003D6C696E6520244A3D6C696E6520245320
:1001F0004C50202443202458202448207E202120B5
:100200003F206374726C2D785D0D0A00536C656538
:1002100070696E6700526573746F72696E672073E0
:1002200070696E646C6500526573746F72696E6795
:100230002064656661756C74730050676D20456E4F
:100240006400436865636B204C696D697473004397
:100250006865636B20446F6F720044697361626C00
:10026000656400456E61626C656400436175746924
:100270006F6E3A20556E6C6F636B6564002724487F
:10028000277C2724582720746F20756E6C6F636B52
:1002900000526573657420746F20636F6E74696EAD
:1002A0007565005B4D53473A00414C41524D3A0051
:1002B0007C413A007C4F763A007C57434F3A007CB1
:1002C000506E3A007C46533A007C42663A007C57B6
:1002D000506F733A007C4D506F733A00536C6565F4
:1002E0007000446F6F723A00436865636B00416C45
:1002F00061726D00486F6D65004A6F6700486F6CF2
:10030000643A0052756E0049646C65000D0A005B2A
:100310005052423A006572726F723A006F6B0D0A6A
:10032000000011241FBECFEFD8E0DEBFCDBF27E015
:10033000A0E0B1E001C01D92A136B207E1F70E9432
:10034000A5010C948C3B0C940000CF93DF93CDB7A8
:10035000DEB762970FB6F894DEBF0FBECDBF8091B7
:10036000C00082608093C0001092C50080E180933D
:10037000C4008091C10088698093C10080E090E052
:100380000E946A288A3009F03DC545E550E061E0E9
:1003900070E08BE291E00E947228892B09F432C54B
:1003A0008AB18C618AB9209A8AB1806E8AB98091AB
:1003B00081008F7E8093810080918100886080938E
:1003C0008100809180008C7F8093800080918000EC
:1003D0008F708093800080916E00887F80936E0084
:1003E00014BC15BC80916E00816080936E0087B153
:1003F000887F87B988B1876088B980916C008760F1
:1004000080936C00809168008260809368008CE02B
:10041000E1E0F1E0DF011D928A95E9F7789410920E
:100420001A018091700184FF03C081E080931A015A
:10043000ADE0CA2EA1E0DA2EB2E0EB2E80911A01D7
:1004400091E1EAE1F1E011929A95E9F780931A01BE
:1004500084E68093210180932201809323018CE024
:10046000D6011D928A95E9F71092190110923B0569
:1004700010923C0510923D0510923E058091FA01C4
:100480008093FB0180E4E0E8F1E011928A95E9F7BE
:1004900064EA71E080E00E94B828811103C087E01F
:1004A0000E94D61E0E94C0343B9A43980E94EB20C3
:1004B0003D98459A80E00E94B21D0E94CA260E9483
:1004C00012320E9433210E94F3348AE591E00E94A7
:1004D000C31E8091700183FF11C00E94CB2088232E
:1004E00069F081E080931A0183EA92E00E94C31EC2
:1004F00082E492E00E94C31E0E946D2080911A0146
:100500008178A1F083EA92E00E94C31E8DE792E019
:100510000E94C31E0E946D2081E080931A0100E0BA
:1005200010E0E3E02E2EF4E03F2E29C010921A01D5
:100530000E94EA1EF4CFE92FF0E0EF5DF94F8081D1
:100540009F5F913809F490E09093FB018F3FE9F0B1
:100550008A3021F50E947B3380911B0181116ECF7F
:10056000E02FF0E0EF5EF84F1082F12FF170FF2ED8
:1005700010FF18C08BE00E94D61E00E010E09091A2
:10058000FB018091FA018913D6CF0E9445320E9467
:100590007B3380911B01882391F350CF8D3009F07C
:1005A00009C4D8CF80911107882309F400C484328C
:1005B00009F0F5C321E0298B80911207833409F1FA
:1005C00034F4882361F0843209F006C11AC08A34F9
:1005D00059F08835B1F0873409F0FEC012C082ECC2
:1005E00091E00E94C31ED9C380911A018F7D09F04A
:1005F000C4C3809113078D3309F0C7C30E940B0752
:10060000BFC3909113079111C0C3833409F4B2C0E2
:100610001CF4843239F0C1C3873469F0883509F499
:10062000C9C0BBC380911A018871F82E09F0A5C317
:100630000E945B1FB2C38CEB91E00E94C31E8091AD
:1006400080018C3838F088EB91E00E94C31E8091C5
:1006500080018A580E949D1E89EA91E00E94C31E73
:10066000809186018A5C0E949D1E89EA91E00E9429
:10067000C31E809184018F5E0E949D1E89EA91E0D5
:100680000E94C31E8091820195E1981B892F0E94D0
:100690009D1E89EA91E00E94C31E80918301865AC3
:1006A0000E949D1E89EA91E00E94C31E80918101F3
:1006B000AEE5A81B8A2F0E949D1E8091870188238A
:1006C00099F08CEA91E00E94C31E809187018330EB
:1006D00029F08E3139F0823039F404C080E30E9471
:1006E000773202C00E949D1E8CEA91E00E94C31ED8
:1006F00080918901803131F0803231F0811107C061
:1007000085E303C083E301C084E30E9477328CEA6F
:1007100091E00E94C31E80918801882311F088E334
:1007200001C089E30E94773285EB91E00E94C31EED
:10073000809193010E949D1E82EB91E00E94C31E56
:1007400060918F017091900180919101909192013F
:100750000E94621E8FEA91E00E94C31E60918B018D
:1007600070918C0180918D0190918E0140E00E94EA
:10077000C41D0EC080911A01823069F40E94F934C0
:1007800083EA92E00E94C31E8AE592E00E94C31EA3
:100790000E946D2002C38111F0C2E0921A0183EA27
:1007A00092E00E94C31E83E692E00E94C31E0E9454
:1007B0006D203BC080911A01813009F0EEC283EABE
:1007C00092E00E94C31E8BE692E00E94C31E0E942C
:1007D0006D2010921A01E1C290911A01923008F036
:1007E000CCC2893409F49FC034F4833271F0883468
:1007F00009F45AC040C1823509F4E7C0833509F4D1
:1008000080C08E3409F037C110C180911307811167
:10081000BCC210E0BE016F5F7F4F812F0E94B828DD
:10082000811105C087E00E94D61EF12CB6C286EA6F
:1008300091E00E94C31E163029F0173041F480EA7F
:1008400091E002C083EA91E00E94C31E04C086E3E7
:10085000810F0E949D1E8AE30E947732CE0101968D
:100860000E94801E0E946D201F5F183099F68AE951
:1008700091E00E94C31E80EB91E00E94801E0E94C6
:100880006D2084E991E00E94C31E6091BC017091CB
:10089000BD018091BE019091BF010E94711E0E9416
:1008A0006D200E94722079C28091700184FF62C223
:1008B00030921A0180911307811167C20E94E020D3
:1008C00084E00E949E2483E00E949E240E947B3349
:1008D00080911B01811106C00E94F3340E943321D4
:1008E0000E94EB2080911B01811157C210921A01C6
:1008F0000E94F4148091130781114FC20E94EA1ED6
:1009000094CF809113078C3409F03FC28091140773
:10091000803509F03AC280911507811136C280E80E
:100920000E94DA1C3AC2E98A80911307811130C013
:1009300040E550E06EEA73E081E197E00E947228A2
:10094000892B51F41092110740E550E061E177E006
:100950008EEA93E00E94DB2680E891E00E94C31EAD
:100960000E94891C0E946D208AE791E00E94C31EAC
:1009700086E50E9477328CE20E9477328FE00E94F7
:100980009D1E8CE20E94773280E80E949D1E00CF5F
:10099000298A8D3309F0F9C183E0282F30E0F9016D
:1009A000EF5EF84F9081D901A25FB84F9C938F5FA3
:1009B00090819111F2CF898B40E550E061E177E0C1
:1009C0008EEA93E00E94DB26E8C18091130783350D
:1009D00009F0DBC180911407843509F0D6C18091FC
:1009E00015078D3309F0D1C1809117078111CDC151
:1009F00080911607843239F08A3239F0833209F057
:100A0000C4C182E003C081E001C08FEF0E94432790
:100A100083EA92E00E94C31E87E292E00E94C31E16
:100A20000E946D200E94F934B8C1E98A80911307B1
:100A300081111DC010E0812F0E94961C811104C0FD
:100A400087E00E94D61E0EC087E791E00E94C31E79
:100A5000812F0E949D1E8DE30E9477320E94891C87
:100A60000E94D21E113009F498C111E0E4CF911117
:100A700084C111E001C010E0BE01635F7F4FCE0171
:100A800041960E940B36811103C072E0F72E85C19A
:100A9000E98981E08E0F898BF0E0EF5EF84F90815D
:100AA0009D3309F072C1112379F1482F50E0282FAE
:100AB00030E0F901EF5EF84F9081241B350BD9012E
:100AC000AF5EB84F9C938F5F90819111F0CF898B6F
:100AD0000E940B07811154C16D857E858F85988991
:100AE0000E94F73A0E9435386A8B0E9487346A89DF
:100AF000B1E56B9FC001112440E550E061E177E072
:100B00009D5F0E94DB2691CEBE016F5F7F4FCE01BD
:100B100041960E940B36882309F4B7CFE989F0E0AB
:100B2000EF5EF84F8081811130C18D849E84AF8447
:100B3000B88820E030E04FE753E4C501B4010E94DB
:100B4000D43918160CF421C149805A806B807C80FE
:100B5000C501B4010E943538062F20E030E0A9011C
:100B6000C301B2010E94B23787FD0CC1043608F4FC
:100B700040C0045680E0033098F510E0000F111FCC
:100B8000000F111F823079F0F801833011F18130AC
:100B900019F0E55DFE4F02C0E95CFE4F40825182D4
:100BA00062827382E4C00D5B1E4F20E030E040E7BC
:100BB00052E4C301B2010E94143A20E030E040E761
:100BC00052E40E94143AF801608371838283938314
:100BD000CEC0E15BFE4F77FA709477F87094DECF69
:100BE0008F5F0A3008F4D1C0843009F4CEC00A50B7
:100BF000C2CFC301B2010E94F73A0E94353810E01B
:100C00000132110508F0C1C0F801EC5CFF4F0C94F3
:100C10005F3B633008F4BCC060935B01A8C0609385
:100C20005E01A5C060935C0102C060935D010E94FB
:100C3000C4149DC080917001662311F0846095C03A
:100C40008B7F93C080917001662311F080648DC00A
:100C50008F7B8BC080917001662311F0806801C08A
:100C60008F778093700180E00E94B21D80C06093F6
:100C70005F017DC04092600150926101609262010B
:100C80007092630174C04092640150926501609259
:100C90006601709267016BC080917001662311F04C
:100CA000816001C08E7F809370010E94661D5FC0CD
:100CB00080917001662321F084FF6DC0806255C071
:100CC0008F7D53C080917001662311F0886001C050
:100CD000877F809370010E94EB2049C08091700152
:100CE000662311F0806141C08F7C3FC06093710129
:100CF0003EC04092720150927301609274017092F2
:100D0000750135C04092760150927701609278016A
:100D1000709279012CC070E070937B0160937A012E
:100D200026C040927C0150927D0160927E017092BB
:100D30007F011DC0409268015092690160926A0172
:100D400070926B0108C040926C0150926D016092EC
:100D50006E0170926F010E94C03409C080917001D1
:100D6000662311F0826001C08D7F809370010E9424
:100D70001A2713C055E0F52E10C048E0F42E0DC020
:100D8000F82E0BC034E0F32E08C023E0F22E05C08D
:100D900096E0F92E02C08AE0F82E8F2D08C08091CF
:100DA0001A01817211F089E0E6CB0E940B070E94C4
:100DB000E21EE3CB112329F0893209F0E0CB1D7F3D
:100DC000DECB813208F4DBCB8F3209F4D8CB88320A
:100DD00099F08B3399F00F3498F4202F30E0E1E054
:100DE000E00F9FE9980FD901AF5EB84F9A3108F430
:100DF00080528C930E2FC3CB12E0C1CB14E0BFCB3B
:100E000011E0BDCB87E00E94D61E8FEF0E944327E2
:100E10000E945B1FC5CA2F923F924F925F926F92C2
:100E20007F928F929F92AF92BF92CF92DF92EF927A
:100E3000FF920F931F93CF93DF93CDB7DEB7CA54C2
:100E4000D1090FB6F894DEBF0FBECDBF8AE3E0EC48
:100E5000F1E0DF011D928A95E9F78BE0E0E8F1E02F
:100E6000A1ECB1E001900D928A95E1F78091110714
:100E7000843211F00C94A61481E08093C101109289
:100E8000C20183E08A8FB1E0BBA3212C312C18AAC8
:100E90001FA6C12C1B8E1F8EDD24D3946AE0A62EC4
:100EA000B12C0EE571E6872E73E0972E8A8DE82F20
:100EB000F0E0EF5EF84FE080EE2009F43EC29FEBD9
:100EC0009E0D9A3110F00C9472148F5F8A8FBE01C0
:100ED0006A5E7F4FCE014A960E940B36882311F43A
:100EE0000C9474144E885F88688C798CC301B201AD
:100EF0000E94F73A0E943538162F70E080E090E0AB
:100F00000E9466389B01AC01C301B2010E94BC364D
:100F100020E030E048EC52E40E94143A0E94813A0A
:100F20000E943538CB01E7E4EE1629F0FDE4EF1618
:100F300009F4EAC034C1183209F4C5C020F51431EF
:100F400068F4113108F08AC0143009F452C008F472
:100F500064C01A3009F445C00C9482141C3109F4A1
:100F600040C050F4163110F00C94821425E1211B7E
:100F70002093C30126E0ACC01E3199F1163209F46A
:100F80004CC00C9482141D3309F497C0A8F4153397
:100F900081F140F41B3209F47AC0113309F477C0AF
:100FA0000C9482141C3310F00C9482146AEC610FC0
:100FB0006093C70129E08CC01C3538F41A3508F05D
:100FC00053C0103581F10C9482141C3551F01F353B
:100FD00010F00C948214202F211B2093C20125E0D5
:100FE00077C0009731F42F8D21110C94761431E0E5
:100FF0003F8F1093C001212F2D7F2C3119F01C350C
:1010000009F063C0009721F00A9711F00C94821444
:10101000610F6093C00120E060C06F8D61110C947E
:101020007614A2E0AF8F1093C101163209F04FC0C1
:101030008431910559F08E31910541F08832910546
:1010400029F08233910511F00C948214B5010E94AD
:10105000293B66576093C10121E03FC06FEE610FED
:101060006093C50122E034C0892B31F466EA610F38
:101070006093C40123E031C06A30710511F00C9413
:1010800082141A3511F40C94821424E026C0BF8D0A
:10109000B1110C947614113331F41092C60128E08A
:1010A000E3E0EF8F1AC00A9711F00C948214D092EB
:1010B000C60128E0F3E0FF8F10C0892B11F00C94DB
:1010C00082142AE00AC027E003C020E001C021E02A
:1010D000892B19F087E10C94AA1481E090E002C0FA
:1010E000880F991F2A95E2F72FA538A928233923BD
:1010F000232B19F085E10C94AA142FA538A9282BCD
:10110000392B38AB2FA7D2CE892B21F7163018F404
:10111000133058F016C0183010F40C9482141A30A2
:10112000F0F01E3159F00C948214112319F0113093
:1011300001F104C033E03093C8011BC01093C80113
:1011400018C0143021F0153031F080E101C080E288
:101150008093CA0102C01092CA018CE00BC0193002
:1011600021F080E48093C90102C01092C9018DE092
:1011700001C08BE0A1E0B0E002C0AA0FBB1F8A95BE
:10118000E2F72FA538A92A233B23232B09F0B2CF5E
:10119000EFA5F8A9EA2BFB2BF8ABEFA787CE8E2D96
:1011A000EE0C990BAA0BBB0BFC01E654F109E531DF
:1011B000F10510F00C948214EB5AFF4F0C945F3B36
:1011C0004092CC015092CD016092CE017092CF013D
:1011D00080E08DC04092D0015092D1016092D20146
:1011E0007092D301FC2DF160CF2E81E080C040923F
:1011F000D4015092D5016092D6017092D7012C2D66
:101200002260C22E82E073C04092D8015092D90170
:101210006092DA017092DB013C2D3460C32E83E0D2
:1012200066C01093DC0184E062C0C301B2010E9479
:101230002E386093DD017093DE018093DF0190937F
:10124000E00185E054C04092E1015092E2016092D9
:10125000E3017092E40186E04AC04092E5015092B9
:10126000E6016092E7017092E80187E040C0409299
:10127000E9015092EA016092EB017092EC0188E082
:1012800036C020E030E04FE753E4C301B2010E94D2
:10129000D439181614F40C9478141093ED0189E0E5
:1012A00026C04092EE015092EF016092F0017092E0
:1012B000F1016B8D61606B8F8AE019C04092F20181
:1012C0005092F3016092F4017092F5018B8D82606F
:1012D0008B8F8BE00CC04092F6015092F701609228
:1012E000F8017092F9019B8D94609B8F8CE0EE2445
:1012F000E394F12C082E02C0EE0CFF1C0A94E2F7D6
:10130000970122213321232B11F00C947A14D4015C
:1013100002C0B595A7958A95E2F7A0FF0BC020E023
:1013200030E0A901C301B2010E94B23787FF02C0B9
:101330000C947C142E283F28B9CDBB8DBB2329F0FB
:10134000EF8DE11102C0F2E0FF8F25FE0FC080910A
:10135000DD019091DE01A091DF01B091E0018138C3
:101360009649A849B10514F00C947E143BA133238F
:1013700001F120FC02C00C9488148091C3018130DB
:1013800009F03FC023E333E34BEC51E46091CC011F
:101390007091CD018091CE019091CF010E94143ABD
:1013A0006093CC017093CD018093CE019093CF01D7
:1013B00028C08091C201813071F46F8D623009F5CF
:1013C0008091C1018035E9F08823D9F020FC02C06A
:1013D0000C94881416C080918101811112C020FCE8
:1013E000CCCF80918F0190919001A0919101B0910B
:1013F00092018093CC019093CD01A093CE01B09344
:10140000CF0130FC10C080918B0190918C01A09194
:101410008D01B0918E018093E9019093EA01A09330
:10142000EB01B093EC018091C001843039F426FCCB
:1014300003C08CE10C94AA14E89426F88091C501AD
:10144000882369F0813029F48BAF1DAA92E09BAB11
:101450000BC01BAEA2E0ADABB1E0BBAB05C0E2E0A0
:10146000EBAFF1E0FDAB1BAA8091C301813021F00D
:101470002F8D2330A9F52BC04EEEE42E41E0F42E43
:1014800000E010E03B8DA32EB12CC501002E02C060
:10149000959587950A94E2F780FF10C023E333E324
:1014A0004BEC51E4D7016D917D918D919C910E94FF
:1014B000143AF70160837183828393830F5F1F4F18
:1014C000F4E0EF0EF11C03301105F9F6D1CF809155
:1014D000C601813029F42B8D243011F00C94801436
:1014E0008CE0E4EAF1E0DE01119601900D928A951C
:1014F000E1F78FA598A991FD09C09091C0019FA324
:101500009A30C9F09C3509F4AFC010C18091C70171
:10151000873018F08DE10C94AA14909186019817E9
:1015200061F3BE016F5F7F4F0E94B828882311F4DA
:101530000C949614E2CFAB8DA11103C08AE10C94F8
:10154000AA14C10180759927892B09F472CF609183
:10155000E1017091E2018091E3019091E4010E9428
:10156000F73A0E9435386730A8F68091DC01843163
:1015700041F0823011F00C94821427FE02C00C94CA
:101580008214BFEA2B22662319F061506DA703C0B5
:10159000E091C701EDA760ED71E08DA50E94B8282C
:1015A000882311F40C949614D090DC014090BC0177
:1015B0005090BD016090BE017090BF0100ED11E040
:1015C00038E9A32E31E0B32EE12CF12CFB8D8F2EC8
:1015D000912CC4010E2C02C0959587950A94E2F7D0
:1015E00080FF34C024E1D21228C0D50158962D9135
:1015F0003D914D915C915B976D917D918D919C9109
:101600000E94BC36F801268D378D40A151A10E9461
:10161000BC36D8016D937D938D939C931397B2E064
:10162000EB16F10499F4A30192010E94BC36F80173
:10163000608371838283938309C0F801868D978DBF
:10164000A0A1B1A180839183A283B383FFEFEF1A9E
:10165000FF0A0C5F1F4F24E0A20EB11C33E0E3161B
:10166000F10409F0B6CF2FC16B8D662309F466CF64
:101670004090BC015090BD016090BE017090BF01D0
:101680000EEE11E0A12CB12CE12CF12C862E912C28
:10169000F501E058FE4FC4010E2C02C095958795C8
:1016A0000A94E2F780FF2BC0A1E0B0E0AC0FBD1FB1
:1016B000AA0DBB1D2D913D914D915C91608D718D59
:1016C000828D938D0E94BC36D8012D913D914D9114
:1016D0005C910E94BC36F80160837183828393839E
:1016E000F2E0EF16F104A1F4A30192010E94BC36CE
:1016F000D8016D937D938D939C93139709C080A916
:1017000091A9A2A9B3A9F80180839183A283B3838D
:10171000FFEFEF1AFF0A24E0A20EB11C0C5F1F4F6F
:1017200033E0E316F10409F0B3CFCCC06F8D633022
:1017300071F48FA18E3109F48BC0853309F4BCC0DC
:101740008C3109F0BFC060ED71E086E084C09B8DF4
:10175000992379F3D090C4014090BC015090BD0111
:101760006090BE017090BF0128E9A22E21E0B22E48
:101770000EEE11E0DE0111964D01E12CF12CE92F66
:10178000F0E0FEA7EDA78DA59EA50E2C02C09595B5
:1017900087950A94E2F780FD0BC0F5018081918165
:1017A000A281B381F80180839183A283B3833FC078
:1017B000FFA1F533E1F1D11029C0D50158962D9143
:1017C0003D914D915C915B97F401608171818281C3
:1017D00093810E94BD36D8012D913D914D915C9130
:1017E0000E94BD36F8016083718382839383F2E0A7
:1017F000EF16F104E1F4A30192010E94BD36D80175
:101800006D937D938D939C93139711C0F501208167
:10181000318142815381D8016D917D918D919C914F
:101820000E94BD36F8016083718382839383FFEF4A
:10183000EF1AFF0A24E0A20EB11C0C5F1F4F34E028
:10184000830E911C63E0E616F10409F09CCF71CF82
:1018500060ED71E087E00E94B828882311F40C94B1
:1018600096148B8D811103C01DA61F8E2CC020E005
:1018700030E080E090E0AB8D4A2F50E0BA01082EB6
:1018800002C0759567950A94E2F760FD0EC0F901F4
:10189000E058FE4F808C918CA28CB38CF901E054FF
:1018A000FE4F808A918AA28AB38A01962C5F3F4FAD
:1018B0008330910519F706C08091C101823010F084
:1018C0000C9484141DA6B091C101BFA3B03529F4B6
:1018D000EB8DE1110C94861474C2FF8DF23009F087
:1018E00070C22FA1211104C03B8D31116AC22BC0DF
:1018F00020E030E0A9016091CC017091CD01809190
:10190000CE019091CF010E94B237882311F40C943C
:1019100088146FA16C3809F43EC240F46230A9F01B
:101920006330B1F0613009F04CC20AC08FA18E382B
:1019300009F431C208F42CC28F3809F429C241C21B
:101940009B8D91113EC21F8E3CC2ABA1A460ABA384
:10195000BB8DBB2309F4F2CDEBA90E2F10E03DA9FE
:10196000232F30E03AA729A781E090E07C010DA861
:1019700002C0EE0CFF1C0A94E2F702C0880F991F08
:10198000EA95E2F7E82AF92A8B2F90E08E219F2131
:10199000892B09F4BFC7F801EE0FFF1FEE0FFF1FE1
:1019A000E054FE4FD801AA0FBB1FAA0FBB1FA856B9
:1019B000BE4F2D913D914D915C9166A577A580A973
:1019C00091A90E94BC364B015C01E9A5FAA5EE0F76
:1019D000FF1FEE0FFF1FE054FE4FA9A5BAA5AA0FE7
:1019E000BB1FAA0FBB1FA856BE4F2D913D914D9115
:1019F0005C9166A577A580A991A90E94BC366FABC2
:101A000078AF89AF9AAF310160E86622772427FE6C
:101A1000EFC0E89427F84CE050E06EEE71E088E902
:101A200091E00E947F3B892B11F481E293C7809162
:101A3000C3018130B1F423E333E34BEC51E4609113
:101A4000E5017091E6018091E7019091E8010E9423
:101A5000143A6093E5017093E6018093E701909357
:101A6000E8014090E5015090E6016090E701709038
:101A7000E801A5019401C501B4010E94143A23961E
:101A80006CAF7DAF8EAF9FAF23972FA938AD49AD17
:101A90005AADCA01B9010E94143A27966CAF7DAFC6
:101AA0008EAF9FAF279720E030E040E850E4C301BD
:101AB000B2010E94143AA30192010E94143A2396A3
:101AC0002CAD3DAD4EAD5FAD23970E94BC36279641
:101AD0002CAD3DAD4EAD5FAD27970E94BC366B017E
:101AE0007C0120E030E0A9010E94B23787FD14C7D5
:101AF000C701B6010E94B33A6B017C0127962CAD59
:101B00003DAD4EAD5FAD279723966CAD7DAD8EADEF
:101B10009FAD23970E94BD360E94B33A9B01AC0152
:101B2000C701B60190580E94BC376B017C018FA1A0
:101B3000833021F4F7FAF094F7F8F09420E030E0E5
:101B4000A901C301B2010E94B23787FF0FC0F7FAA3
:101B5000F094F7F8F094D301C201B0588093E501F6
:101B60009093E601A093E701B093E801000F111FE5
:101B7000000F111F00531E4FA70196016FA978ADEA
:101B800089AD9AAD0E94143A9B01AC01C501B40124
:101B90000E94BC3620E030E040E05FE30E94143A4F
:101BA000D8016D937D938D939C93139709A51AA5E6
:101BB000000F111F000F111F00531E4FA7019601A8
:101BC000C501B4010E94143A9B01AC016FA978AD24
:101BD00089AD9AAD0E94BD3620E030E040E05FE381
:101BE0000E94143AF8016083718382839383E9C071
:101BF000D12CEC20FD20EF2809F490C6F1EF2F2224
:101C00008091C301813009F47CC0F801EE0FFF1F01
:101C1000EE0FFF1FE053FE4FC080D180E280F380C3
:101C2000A7019601C501B4010E94BC362B013C01FD
:101C3000E9A5FAA5EE0FFF1FEE0FFF1FE053FE4FC1
:101C400080819181A281B38189A79AA7ABA7BCA704
:101C50009C01AD016FA978AD89AD9AAD0E94BC36EB
:101C60004B015C01A3019201C301B2010E94143A2D
:101C70002B013C01A5019401C501B4010E94143A55
:101C80009B01AC01C301B2010E94BD360E94B33A70
:101C90004B015C01A7019601C701B6010E94143AED
:101CA0006B017C0129A53AA54BA55CA5CA01B90128
:101CB0000E94143A9B01AC01C701B6010E94BD36D7
:101CC0000E94B33A6B017C016093E5017093E601D9
:101CD0008093E7019093E8019B01AC01C501B40139
:101CE0000E94BC364B015C01E894B7F82AE037ED5E
:101CF00043EA5BE3C501B4010E94D43918165CF1D4
:101D000060C090ECE92E91E0F92EC601062C02C0CD
:101D1000959587950A94E2F780FF12C023E333E399
:101D20004BEC51E4D70150966D917D918D919C9132
:101D300053970E94143AF701608B718B828B938BBF
:101D4000FFEF6F1A7F0A24E0E20EF11C33E0631606
:101D50007104D9F65ACF20E030E040E05FE3C501DE
:101D6000B4010E94D43918160CF45FCE2FE632E18C
:101D700043E85AE3C701B6010E94143A9B01AC0143
:101D8000C501B4010E94D43918160CF44ECE19C006
:101D90006BA160616BA38FA18E58823018F48BA168
:101DA00088608BA39B8D992309F4C8CB4CE050E04D
:101DB0006EEE71E088E991E00E947F3B892B09F487
:101DC00034CE2BA12170ABA1C101A0FF02C08E7D3A
:101DD00002C08E7D9C7FBF8DB111937E892B09F04F
:101DE0009FC58E01035F1F4F89E0F80111928A950C
:101DF000E9F7222309F44BC08FA598A9867B892B8C
:101E000009F090C58091C001853311F081118AC518
:101E100080918B0190918C01A0918D01B0918E01E8
:101E2000898B9A8BAB8BBC8B9091890180918801B7
:101E3000892B4091CC015091CD016091CE017091E0
:101E4000CF014D875E876F87788B84608D8B809103
:101E5000700185FF06C08EEE91E00E94E31C8111A7
:101E600063C5B8018EEE91E00E949F3580911A0102
:101E700081115EC50E94BA26892B09F459C580E2FA
:101E800080931A010E94D9280E94721751C580912F
:101E90007001F090890181FF26C09FA1915093307D
:101EA00018F0FBA1F064FBA32B8D222339F03F8DAA
:101EB000323021F46BA160686BA315C080E1F81289
:101EC00012C09091800191508BA18074933030F4B6
:101ED000882349F09BA190629BA305C0811103C098
:101EE000ABA1A062ABA38091DD019091DE01A09136
:101EF000DF01B091E0018093940190939501A0934C
:101F00009601B09397018091C2018093810188234B
:101F100011F088E08D8B8091CC019091CD01A09142
:101F2000CE01B091CF0180938F0190939001A09347
:101F30009101B09392018D879E87AF87B88B809077
:101F4000E9019090EA01A090EB01B090EC01A501AD
:101F5000940160918B0170918C0180918D01909121
:101F60008E010E94B237BBA1B074EB2E811103C069
:101F7000EBA1E5FF20C0FF2071F0FBA1F7FD0BC036
:101F8000EE2021F040E050E0BA0102C0B501A4010A
:101F90008F2D0E9498348091E9019091EA01A091DF
:101FA000EB01B091EC0180938B0190938C01A09395
:101FB0008D01B0938E01E1100CC080918B01909146
:101FC0008C01A0918D01B0918E01898B9A8BAB8B86
:101FD000BC8B8091ED01809393018091CA01909117
:101FE0008901981751F049895A896B897C890E9427
:101FF00098348091CA01809389019D8980918901DB
:10200000892B8D8B8091C901909188019817D1F00F
:1020100090911A01923051F02B968FAF2B970E941E
:1020200087342B968FAD2B970E9493328091C901F4
:10203000811103C01092880105C090918801892BFD
:10204000809388019D8980918801892B8D8B809157
:10205000C001843049F56091E1017091E201809105
:10206000E3019091E40120911A012230E9F02896D1
:102070006FAF289729967FAF29972B968FAF2B9715
:102080002A969FAF2A970E94873440E028966FAD2A
:10209000289729967FAD29972B968FAD2B972A9657
:1020A0009FAD2A970E9402218091C50180938401EF
:1020B0008091C301809382012F8D233071F580912F
:1020C000C60180938501811108C01092F60110921B
:1020D000F7011092F8011092F901C090F601D0902A
:1020E000F701E090F801F090F901A70196016091E5
:1020F000BC017091BD018091BE019091BF010E9411
:10210000B237882351F0C092BC01D092BD01E09259
:10211000BE01F092BF010E94661D8091C70190919F
:102120008601981769F0809386018CE0FE01319654
:10213000A4EAB1E001900D928A95E1F70E94661D34
:102140008091C401809383018091C0018632F1F1B6
:1021500038F48C3109F18E31F9F08A3069F04FC0D2
:102160008C35D1F1863609F441C0883209F047C078
:1021700068E971E087E02DC060ED71E08DA50E94F7
:102180002727809186013DA5831339C08CE0E0EDBF
:10219000F1E0A4EAB1E025C08D8981608D8B6F8D5F
:1021A000662329F0B8018EEE91E00E949F35B801B8
:1021B00080ED91E00E949F358CE0E0EDF1E0A8E930
:1021C000B1E001900D928A95E1F719C068E971E0DC
:1021D00086E00E94272713C08CE0EEEEF1E0A0EB32
:1021E000B1E001900D928A95E1F707C08CE0E0EB39
:1021F000F1E0DF011D928A95E9F70E94661D80914A
:10220000C10180938001803509F41EC3BF8DB230B7
:1022100009F01AC3813021F4BE01635F7F4F06C00D
:10222000811109C08D8981608D8BB8018EEE91E09E
:102230000E949F3500C38250823008F095C2809181
:10224000E5019091E601A091E701B091E8018F8F3F
:1022500098A3A9A3BAA3ABA994E0A99F70011124E4
:10226000F701E856FE4FF8A7EFA3970120533E4F22
:102270003EA72DA7D9014D905D906D907C90208157
:10228000318142815381C301B2010E94BD366FA7E3
:1022900078AB89AB9AABEDA9B4E0EB9F8001112438
:1022A000980128563E4F3CAB2BABC80180539E4F44
:1022B0009EAB8DABDC018D909D90AD90BC90F901F3
:1022C0002081318142815381C501B4010E94BD3614
:1022D0006FAB78AF89AF9AAF77FA709477F8709454
:1022E000D501C401B0588B8F9C8FAD8FBE8FF70185
:1022F000E251FE4F2FA538A949A95AA960817181E1
:10230000828193810E94BC366B017C01F801E2510D
:10231000FE4F2FA938AD49AD5AAD608171818281E0
:1023200093810E94BC364B015C01A7019601C30159
:10233000B2010E94143A69A77AA78BA79CA7A501AE
:1023400094016B8D7C8D8D8D9E8D0E94143A9B0126
:10235000AC0169A57AA58BA59CA50E94BD3669A78D
:102360007AA78BA79CA7A5019401C301B2010E9483
:10237000143A4B015C01A70196016B8D7C8D8D8D0C
:102380009E8D0E94143A9B01AC01C501B4010E94CC
:10239000BC3629A53AA54BA55CA50E943C376B012C
:1023A0007C019BA192FF13C02DEB37E346E055EB78
:1023B000C701B6010E94D43987FD1DC02BED3FE057
:1023C00049EC50E4C701B6010E94BC3612C02DEBA7
:1023D00037E346E055E3C701B6010E94B23718164D
:1023E00054F02BED3FE049EC50E4C701B6010E94E8
:1023F000BD366B017C018090640190906501A090D6
:102400006601B09067012F8D38A149A15AA1CA0178
:10241000B9010E94BD36A50194010E94BC369B0102
:10242000AC01C501B4010E94143A0E94B33A4B01B9
:102430005C0120E030E040E05FE3C701B6010E94AC
:10244000143A2F8D38A149A15AA10E94143A9F77BE
:10245000A50194010E94BC370E94A1380E94353822
:102460007AA769A7DB01AB2B09F4D6CE1D894B01F6
:10247000A12CB12C13FF12C0C501B4010E94643815
:102480009B01AC016D857E858F8598890E94143AE9
:102490006D877E878F87988B177F1D8BC501B40151
:1024A0000E9464384B015C019B01AC01C701B6017D
:1024B0000E94BC376BA37CA38DA39EA3EBADB4E0BD
:1024C000EB9FC00111248C0108561E4FFC01E25104
:1024D000FE4FD8012D913D914D915C9160817181AC
:1024E000828193810E94BC36A50194010E94BC3771
:1024F00027966CAF7DAF8EAF9FAF27972BA13CA1E6
:102500004DA15EA1CA01B9010E94143A9B01AC0120
:1025100060E070E080E090E40E94BC366B017C01DA
:102520002BEA3AEA4AE25EE36BA17CA18DA19EA16F
:102530000E94143A4B015C0120E030E040E850E496
:10254000C701B6010E94BD369B01AC01C501B401B3
:102550000E94143A6BAF7CAF8DAF9EAF20E030E0AD
:1025600040E05FE3C701B6010E94143A23966CAFC6
:102570007DAF8EAF9FAF23971F8E22242394312CE3
:10258000E9A5FAA52E163F0609F446CEBF8DBC304C
:1025900008F044C023962CAD3DAD4EAD5FAD239702
:1025A0006B8D7C8D8D8D9E8D0E94143A6B017C010C
:1025B0002BAD3CAD4DAD5EADC301B2010E94143AEE
:1025C000A70196010E94BD367B016C0123962CADBC
:1025D0003DAD4EAD5FAD2397C301B2010E94143AE9
:1025E0004B015C012BAD3CAD4DAD5EAD6B8D7C8D7B
:1025F0008D8D9E8D0E94143A9B01AC01C501B401E2
:102600000E94BC362B013C01EF8DEF5FEF8F47013D
:1026100056018B8E9C8EAD8EBE8E65C0B10180E062
:1026200090E00E9464382BA13CA14DA15EA10E94C4
:10263000143A6B017C010E94B7376B8F7C8F8D8FB2
:102640009E8FC701B6010E94A53A4B015C01ADA562
:10265000BEA5CD90DD90ED90FC90F7FAF094F7F8E0
:10266000F094ADA9BEA98D919D910D90BC91A02D26
:102670008F8F98A3A9A3BAA32B8D3C8D4D8D5E8D12
:10268000C701B6010E94143A2B013C01A501940137
:102690006F8D78A189A19AA10E94143A9B01AC0187
:1026A000C301B2010E94BD362B013C01A50194017A
:1026B000C701B6010E94143A6B017C012B8D3C8D41
:1026C0004D8D5E8D6F8D78A189A19AA10E94143ADB
:1026D0009B01AC01C701B6010E94BC366B8F7C8F99
:1026E0008D8F9E8F1F8EA30192016FA578A989A956
:1026F0009AA90E94BD36EFA1F8A5608371838283F9
:1027000093832B8D3C8D4D8D5E8D6FA978AD89ADFA
:102710009AAD0E94BD36ABA9BCA96D937D938D93F4
:102720009C93139727962CAD3DAD4EAD5FAD27978B
:10273000F80160817181828193810E94BD36D80148
:102740006D937D938D939C931397BE01635F7F4F31
:1027500088E991E00E949F3580911B0181116BC037
:10276000BFEF2B1A3B0A0CCF8D8984608D8B809133
:102770001A01823009F45FC00E94873480911B01E6
:10278000811162C0FBA1F071FF2E10921F012BA1DD
:1027900023FB882780F90E94B21D86B18072909138
:1027A0000001891749F084E00E94CA1C0E947B3313
:1027B00080E00E94B21D48C0B8018EEE91E00E94F8
:1027C0009F3581E08093190182E00E94DA1C0E940B
:1027D0007B3380911B01811137C080911A018111D7
:1027E000F6CF80911901813081F4FF2051F08CE007
:1027F000E1E0F1E0ADE0B1E001900D928A95E1F702
:1028000007C085E00E94CA1C03C081E080931F01BD
:102810001092190180E00E94B21D0E947B330E9439
:1028200012320E94CA260E9433210E947220809197
:102830001F01811188C08CE0EEEEF1E0A8E9B1E063
:1028400001900D928A95E1F78091C80180938701EC
:10285000882309F47FC00E9487348091870190917A
:102860001A01833041F49230D1F188E00E94DA1CE1
:102870000E947B3334C081E08093800110928401F8
:1028800010928301109281011092860110928901A9
:102890001092880184E68093210180932201809325
:1028A0002301923091F064EA71E080E00E94B82840
:1028B0008823E1F10E94661D40E050E0BA0180E00B
:1028C0000E94503380E00E94933283EA92E00E949B
:1028D000C31E8AE392E00E94C31E0E946D201092E4
:1028E00087012FC081E036C082E034C088E132C069
:1028F00086E230C089E12EC084E02CC08BE12AC082
:1029000085E228C084E126C08EE124C08FE122C088
:1029100086E120C080E21EC082E21CC083E21AC0B1
:1029200084E218C080E116C08FE014C087E012C0B6
:102930008CE0EEEEF1E0A8E9B1E001900D928A950D
:10294000E1F780E007C00E94F3347ECF1A8E1BA20D
:102950000C944507C65BDF4F0FB6F894DEBF0FBE81
:10296000CDBFDF91CF911F910F91FF90EF90DF903E
:10297000CF90BF90AF909F908F907F906F905F901F
:102980004F903F902F90089580915C01682F90E0C8
:1029900020915D01422F80FD94E0822F817020FD07
:1029A00080E261FD986041FD806462FD906142FDBE
:1029B000806890933F058093400508951F920F9281
:1029C0000FB60F9211248F939F938BB190913F0577
:1029D0009C71837E892B8BB915BC9F918F910F9031
:1029E0000FBE0F901F90189580916F008D7F809380
:1029F0006F0080918100887F8160809381001092B8
:102A0000410580915E0190911A018F3F39F4209128
:102A10003C05211103C0903881F402C0943069F064
:102A200090E0009741F0EFE9FFE03197F1F700C047
:102A300000000197F6CF81E001C080E09091700125
:102A400092FF02C091E08927882311F0289A089507
:102A5000289808951F920F920FB60F9211242F936A
:102A60003F934F935F936F937F938F939F93AF9316
:102A7000BF93EF93FF9380914105811122C28BB1E7
:102A800090915105907E8F71892B8BB98BB1837E8C
:102A900090915005892B8BB980914F0586BD82E0BE
:102AA00085BD81E080934105789480916305909184
:102AB0006405892B09F0BFC0809165059091900550
:102AC000981709F4A4C0E09165052E2F30E087E047
:102AD000E89FF0011124EA59FA4FF0936405E0935E
:102AE000630582819381909389008093880080811F
:102AF000918190935F0580935E05E48180916005EC
:102B00008E1761F1E093600582E1E89FF0011124E6
:102B1000EF56FA4FF0936205E09361058485958541
:102B2000A685B785B695A7959795879580934A050D
:102B300090934B05A0934C05B0934D0580934605AB
:102B400090934705A0934805B093490580934205AB
:102B500090934305A0934405B0934505A09161056A
:102B6000B09162059091400550968C9150978927BD
:102B70008093510587E0829FF001839FF00D11241F
:102B8000EA59FA4F25814D915D916D917C91139792
:102B9000022E04C076956795579547950A94D2F70B
:102BA0004093520550935305609354057093550517
:102BB00014964D915D916D917C911797022E04C0F2
:102BC00076956795579547950A94D2F740935605A1
:102BD00050935705609358057093590518968D9139
:102BE0009D910D90BC91A02D04C0B695A795979589
:102BF00087952A95D2F780935A0590935B05A09309
:102C00005C05B0935D0586810E94423314C00E942A
:102C1000F414E0916105F09162058189882339F00F
:102C20001092B3008091B0008F778093B00084E061
:102C30000E94DA1C46C1809119018130B1F486B13D
:102C4000807290910001891781F0109219018CE037
:102C5000E1E0F1E0ADE0B1E001900D928A95E1F79D
:102C600080913B05806480933B0510925005409114
:102C7000520550915305609154057091550580910E
:102C8000420590914305A0914405B0914505840FFC
:102C9000951FA61FB71F8093420590934305A093ED
:102CA0004405B0934505E0916105F09162054485C6
:102CB000558566857785481759076A077B0768F544
:102CC00024E0209350054485558566857785841BCF
:102CD000950BA60BB70B8093420590934305A093E9
:102CE0004405B0934505208980910101909102012E
:102CF000A0910301B091040125FF04C00197A1092F
:102D0000B10903C00196A11DB11D809301019093EB
:102D10000201A0930301B093040140915605509124
:102D2000570560915805709159058091460590911D
:102D30004705A0914805B0914905840F951FA61F2E
:102D4000B71F8093460590934705A0934805B0931D
:102D500049054485558566857785481759076A076B
:102D60007B0778F520915005286020935005448515
:102D7000558566857785841B950BA60BB70B8093CD
:102D8000460590934705A0934805B09349052089CF
:102D90008091050190910601A0910701B091080171
:102DA00026FF04C00197A109B10903C00196A11D26
:102DB000B11D8093050190930601A0930701B09384
:102DC000080140915A0550915B0560915C05709136
:102DD0005D0580914A0590914B05A0914C05B091FD
:102DE0004D05840F951FA61FB71F80934A0590932A
:102DF0004B05A0934C05B0934D05448555856685DC
:102E00007785481759076A077B0778F520915005A1
:102E10002061209350054485558566857785841B00
:102E2000950BA60BB70B80934A0590934B05A09387
:102E30004C05B0934D0520898091090190910A01BC
:102E4000A0910B01B0910C0127FF04C00197A109CB
:102E5000B10903C00196A11DB11D80930901909392
:102E60000A01A0930B01B0930C0180911A018430E8
:102E700039F4909120018091500589238093500569
:102E800080915E0590915F05019790935F05809317
:102E90005E05892B69F41092640510926305809198
:102EA00065058F5F80936505863011F41092650586
:102EB00090913F058091500589278093500510928D
:102EC0004105FF91EF91BF91AF919F918F917F91BC
:102ED0006F915F914F913F912F910F900FBE0F9087
:102EE0001F9018958091700182FF02C0289A01C03E
:102EF000289880913F058093500580915B01880F51
:102F00008450819580934F0580916F0082608093FB
:102F10006F0008953F924F925F926F927F928F92CF
:102F20009F92AF92BF92CF92DF92EF92FF920F9358
:102F30001F93CF93DF93CDB7DEB7A4970FB6F89466
:102F4000DEBF0FBECDBF10913C05112391F181E092
:102F500080931A0189EA92E00E94C31E812F0E9489
:102F60009D1E0E94D21E85EF91E0019739F0EFE996
:102F7000FFE03197F1F700C00000F7CF1150123099
:102F800030F08FB7F89410923C058FBF12C083EADF
:102F900092E00E94C31E81E992E00E94C31E0E943B
:102FA0006D2080E10E94D01C80913B0584FFFCCF06
:102FB000E8CF10913B05112309F4BEC214FF04C0F1
:102FC00081E080931B01BBC310FFC0C18CE0E1E036
:102FD000F1E0DE01599601900D928A95E1F7BE016C
:102FE000675E7F4FCE010D960E941E1D8CE30E94EE
:102FF000773280911A018830E1F058F4813099F1EC
:10300000A8F0823099F1843009F043C084EF92E057
:103010003EC0803229F118F4803171F03AC080341A
:1030200041F18038B1F58CED92E031C087E093E05A
:103030002EC083E093E02BC080911C0187FD10C05F
:103040008DEF92E00E94C31E80911C0180FF06C09C
:1030500080E31AC082FF17C085FFFACF81E314C056
:1030600089EF92E014C08EEE92E011C088EE92E0FB
:103070000EC082EE92E00E94C31E80911C0183FF6D
:10308000E9CF83E301C082E30E94773202C00E944D
:10309000C31E80915F01F82FF170BF2E80FD15C017
:1030A0004090BC015090BD016090BE017090BF0186
:1030B00044EA842E41E0942E9E012F5F3F4F790118
:1030C000CE010D966C0100E02CC080912601882372
:1030D00039F385ED92E03FC0A30192010E94BD3615
:1030E000F7016083718382839383B110F2CFF7017C
:1030F0002081318142815381F60160817181828119
:1031000093810E94BC36F60160837183828393832E
:103110000F5FF4E0EF0EF11C24E0C20ED11C03306F
:10312000B1F0F40161917191819191914F012085EC
:103130003185428553850E94BD36F70160837183D6
:1031400082839383023041F2BB2089F2E1CFB11038
:10315000C0CF8EEC92E00E94C31ECE010D960E945D
:10316000801E80915F0181FF1FC089EC92E00E9468
:10317000C31E90911E058091FD01981710F0815F8C
:1031800001C08150891B0E949D1E8CE20E947732F3
:103190008091FB019091FA01981710F0805801C0BE
:1031A0008150891B0E949D1E84EC92E00E94C31EE8
:1031B00080911A018C7749F06091020670910306A4
:1031C000809104069091050603C060E070E0CB0199
:1031D0000E94621E8CE20E947732609127017091FA
:1031E00028018091290190912A0140E00E94C41D8C
:1031F0000E94CB20F82E0E946B1D082F86B1982FBD
:10320000907280910001E92EE8268F2D802B8E2967
:1032100059F18FEB92E00E94C31EEE2019F080E579
:103220000E947732FF2079F0F0FE03C088E50E940B
:103230007732F1FE03C089E50E947732F2FE03C0C7
:103240008AE50E947732002379F000FF03C082E50F
:103250000E94773201FF03C088E40E94773202FFA8
:1032600003C083E50E94773280912601882321F0F4
:1032700081508093260118C080911A018C7711F03B
:103280008DE101C089E080932601809125018111A3
:1032900003C081E08093250189EB92E00E94C31E68
:1032A000CE0101960E94801E00912501002321F08D
:1032B00001500093250142C080911A018C7711F0D2
:1032C00083E101C089E08093250184EB92E00E94B4
:1032D000C31E809121010E949D1E8CE20E947732C4
:1032E000809122010E949D1E8CE20E947732809183
:1032F00023010E949D1E8091B00087FF05C02D997B
:1033000002C001E001C002E0439B03C0FF24F3942C
:1033100003C0002399F0F12C80EB92E00E94C31EC1
:10332000002339F0013011F483E501C083E40E94E9
:103330007732FF2019F086E40E9477328EE30E94F4
:1033400077320E94D21E81E00E94D01C812F887E9D
:1033500009F469C080911A01982F937009F052C046
:103360008872A1F080911C01807C81F40E94A830B9
:1033700082E080931E0180911A01803239F417FD9A
:1033800005C080911C01806880931C0180911A0106
:10339000811103C091E090931C0116FF07C085FDC9
:1033A00005C090911C01906490931C0113FF05C00F
:1033B000807E19F480E180931A0115FF23C083EA0F
:1033C00092E00E94C31E8FE492E00E94C31E0E94FE
:1033D0006D2080911C0187FD10C090911A019034DE
:1033E00039F483FF07C0837E826080931C0102C092
:1033F000903819F080E480931A0180911C0180625A
:1034000080931C0117FF0CC080911A01813029F4B0
:1034100080911C01856080931C0180E880931A01D3
:1034200088EE0E94D01C11FF44C0812F8876F1F5F0
:1034300080911A01803471F480911C0185FD0AC0CD
:1034400084FF03C010921A0105C082FF03C0886088
:1034500080931C0180911A01882381F084FF26C08B
:1034600090911C0190FF22C0803141F48091240191
:10347000882321F088608093240118C010921E01D7
:103480000E94BA26892B71F080911C0186FD0AC02A
:1034900010921C0188E080931A010E94D9280E9492
:1034A000721704C010921C0110921A0182E00E944F
:1034B000D01C12FF41C080911A01807D90911C01A7
:1034C0008823D9F080911D01811117C097FD15C087
:1034D0000E94A8308091FD0180931B060E94CC3091
:1034E00080911E0181FF05C090911C019160909315
:1034F0001C01897F80931E011CC097FF0AC0109297
:103500001E010E94CA260E9412320E94F3340E94B9
:10351000332180911C0185FF08C08F7781608093E3
:103520001C0180E480931A0104C010921C011092C7
:103530001A0184E00E94D01C90913D05992309F462
:10354000ABC08FB7F89410923D058FBF4091210119
:1035500090FF02C084E601C0842F91FD865F92FD3A
:103560008A5093FD8F5F94FD8150893C08F088EC70
:103570008A3008F48AE03091220195FF02C024E6E7
:1035800001C0232F96FD22E397FD29E1841303C098
:10359000231709F481C08093210120932201109206
:1035A00025011091FD0130901E0589E9D82E96E77E
:1035B000E92E26E9F22E0EE732E3432E131509F425
:1035C00057C0812E912C489CC001499C900D11241C
:1035D000FC01E250FE4F5F01CF010E945521562EA3
:1035E000672E782EC92E2D2D3E2D4F2D502F0E9447
:1035F000D43918164CF42D2D3E2D4F2D502F6D2DF6
:103600007E2D8F2D902F08C0252D362D472D5C2D1A
:10361000652D762D872D9C2D0E94143AF501668B21
:10362000778B808F918F489CC001499C900D11240D
:103630009C0122503E4F7901F90182A093A0A4A0E1
:10364000B5A0A501940166897789808D918D0E942E
:10365000D43918162CF4F701868A978AA08EB18E79
:103660001F5F103109F410E0D52C73010C2DA6CF8B
:103670008D2D9E2DAF2DB02F80933705909338055B
:10368000A0933905B0933A050E94A8308091FD01BE
:1036900080931B060E94CC3090913E05992309F43B
:1036A00048C08FB7F89410923E058FBF2091230138
:1036B00090FF02C084E601C0822F91FD865F92FDDB
:1036C0008A5093FD8F5F94FD8150893C08F088EC0F
:1036D0008A3008F48AE0821749F020911E012860A0
:1036E00020931E01809323011092250180911A01DD
:1036F00095FF0DC0803159F420912401211102C0A1
:1037000022E003C020FF03C0246020932401907CAA
:1037100081F0882311F0887161F01091880116FF03
:1037200002C01F7B01C01064812F0E94933210934E
:10373000880180911A018C7F11F00E94D928A496EB
:103740000FB6F894DEBF0FBECDBFDF91CF911F91B2
:103750000F91FF90EF90DF90CF90BF90AF909F9030
:103760008F907F906F905F904F903F9008956F92F1
:103770007F928F929F92AF92BF92CF92DF92EF9201
:10378000FF920F931F93CF93DF93EB018C015B01AB
:103790008CE0A80EB11C89E9682E96E7792E26E9FF
:1037A000822E3EE7932EC990D990E990F99020E0BF
:1037B00030E0A901C701B6010E94B2378823B9F0F1
:1037C000A7019601F80160817181828193810E9435
:1037D000BC376B017C01E894F7F8A7019601B301AF
:1037E000C4010E94B23787FD02C0360147010C5F59
:1037F0001F4FCA15DB05B9F6B301C401DF91CF91A4
:103800001F910F91FF90EF90DF90CF90BF90AF90FE
:103810009F908F907F906F9008954F925F926F92DC
:103820007F92AF92BF92CF92DF92EF92FF920F936F
:103830001F93CF93DF93EC018C015C018CE0A80E09
:10384000B11CC12CD12C7601F801419051906190AE
:1038500071908F0120E030E0A901C301B2010E9404
:10386000B237882371F0A3019201C301B2010E9413
:10387000143A9B01AC01C701B6010E94BD366B0131
:103880007C010A151B0501F7C701B6010E94B33A76
:103890002B013C019B01AC0160E070E080E89FE3FC
:1038A0000E94BC376B017C019B01AC01688179816E
:1038B0008A819B810E94143A688379838A839B83DF
:1038C000A70196016C817D818E819F810E94143AAF
:1038D0006C837D838E839F83A7019601688579859C
:1038E0008A859B850E94143A688779878A879B8797
:1038F000C301B201DF91CF911F910F91FF90EF9023
:10390000DF90CF90BF90AF907F906F905F904F907F
:103910000895CF93DF93C1E1D7E08991882319F00F
:103920000E947732FACFDF91CF910895CF93DF9342
:1039300021E5829FC0011124EC01DD5F40E550E0EC
:10394000BE0181E197E00E947228892B69F41092F0
:1039500011070E94873440E550E061E177E0CE0135
:103960000E94DB2680E001C081E0DF91CF910895C5
:103970002FB7F89490913E05892B80933E052FBF79
:1039800008952FB7F89490913D05892B80933D05BC
:103990002FBF08959FB7F89480933C059FBF08956B
:1039A0002FB7F89490913B058095892380933B0530
:1039B0002FBF08952FB7F89490913B05892B8093E2
:1039C0003B052FBF0895AF92BF92CF92DF92EF9247
:1039D000FF920F931F93CF93DF93EC010FE411E05D
:1039E0005C018CE0A80EB11CC990D990E990F990C7
:1039F00020E030E0A901C701B6010E94D4391816B1
:103A00008CF0F80121913191419151918F01C701C1
:103A1000B6010E94B23787FD05C0CA15DB0521F744
:103A200080E001C081E0DF91CF911F910F91FF9065
:103A3000EF90DF90CF90BF90AF900895AF92BF927C
:103A4000CF92DF92EF92FF920F931F93CF93DF936A
:103A500000D000D0CDB7DEB75B012BE2E22E21E033
:103A6000F22E8C016B018CE0C80ED11CF501619126
:103A70007191819191915F01F70121913191419172
:103A800051917F0129833A834B835C830E9466387E
:103A900029813A814B815C810E94BC37F801619396
:103AA0007193819391938F01AC14BD04F9F60F903B
:103AB0000F900F900F90DF91CF911F910F91FF907A
:103AC000EF90DF90CF90BF90AF9008950E94873421
:103AD00010922601089596B1892F877049F0892F99
:103AE0008095817091FF826092FD03C0846008958B
:103AF00080E008951F920F920FB60F9211242F931A
:103B00003F934F935F936F937F938F939F93AF9365
:103B1000BF93EF93FF930E946B1D882391F080FF6A
:103B200003C00E94F9340DC082FF04C080913B05A0
:103B3000826005C081FF05C080913B05886080934D
:103B40003B05FF91EF91BF91AF919F918F917F9135
:103B50006F915F914F913F912F910F900FBE0F90FA
:103B60001F901895109200019091700197FD03C06D
:103B700090E290930001882331F09091000180E25F
:103B800089278093000108958F929F92AF92BF92F0
:103B9000CF92DF92EF92FF920F931F93CF93DF9319
:103BA000CDB7DEB72D970FB6F894DEBF0FBECDBFF1
:103BB0006B017C01042F20E030E0A9010E94B237A4
:103BC00087FF07C08DE20E947732F7FAF094F7F88A
:103BD000F094102F123060F020E030E048EC52E416
:103BE000C701B6010E94143A6B017C011250F2CF5A
:103BF00000FF0AC020E030E040E251E4C701B60116
:103C00000E94143A6B017C0120E030E040E05FE369
:103C1000C701B6010E94BD360E942E3810E03AE07E
:103C2000832E912CA12CB12C611571058105910574
:103C300091F0EE24E394F12CEC0EFD1EE10EF11C4C
:103C4000A50194010E943D3B605DF7016083B901CD
:103C5000CA011F5FE9CF80E3101748F4E1E0F0E00C
:103C6000EC0FFD1FE10FF11D80831F5FF5CF1013D7
:103C700014C011E0100F80E3FE01E00FF11D8183FD
:103C80000CC0101303C08EE20E947732FE01E10FD8
:103C9000F11D80810E94773211501111F2CF2D96C3
:103CA0000FB6F894DEBF0FBECDBFDF91CF911F914D
:103CB0000F91FF90EF90DF90CF90BF90AF909F90CB
:103CC0008F9008952091700120FF08C02BE832E406
:103CD00041E25DE30E94143A41E001C040E00C94EF
:103CE000C41D2091700120FF08C02BE832E441E29E
:103CF0005DE30E94143A44E001C043E00C94C41D0B
:103D0000CF93DF93EC01688179818A819B810E9446
:103D1000711E8CE20E9477326C817D818E819F8141
:103D20000E94711E8CE20E947732688579858A85AF
:103D30009B85DF91CF910C94711ECF93DF938436D6
:103D400030F06AE00E941D3BC0E3C90F03C0C0E031
:103D50008A3030F06AE00E941D3BD0E3D90F01C0E9
:103D6000D0E0805D0E947732DD2319F08D2F0E9414
:103D70007732CC2329F08C2FDF91CF910C947732BE
:103D8000DF91CF910895CF93DF93FC018491EF01F0
:103D90002196882321F00E947732FE01F7CFDF9130
:103DA000CF9108958CE093E00C94C31ECF93C82F5D
:103DB00085E193E00E94C31E8C2F0E949D1ECF912F
:103DC0000C94D21E811104C08CE193E00C94C31EAC
:103DD0000C94D61ECF93DF93C0E08C2F0E94961CCC
:103DE00081110EC0109211078EE30E9477320E945B
:103DF000891C8AE30E94773287E00E94D61E12C097
:103E000080911107882371F00E940B07D82F8EE351
:103E10000E9477320E94891C8AE30E9477328D2F9C
:103E20000E94E21EC13011F0C1E0D7CFDF91CF91E7
:103E30000895CF92DF92EF92FF921F93CF93DF937B
:103E40001F92CDB7DEB7182F6A017B0184E2298368
:103E50000E947732812F0E949D1E8DE30E9477324F
:103E60002981422FC701B6010E94C41D0F90DF9126
:103E7000CF911F91FF90EF90DF90CF900C94D21EC6
:103E80001F93CF93DF931F92CDB7DEB7182F84E235
:103E900069830E947732812F0E949D1E8DE30E94CC
:103EA00077326981862F0E949D1E0F90DF91CF91FE
:103EB0001F910C94D21EEF92FF920F931F93CF93FA
:103EC000DF9360915B0170E080E00E94401F609191
:103ED0005E0170E081E00E94401F60915C0170E033
:103EE00082E00E94401F60915D0170E083E00E94CB
:103EF000401F6091700162FB662760F970E084E00A
:103F00000E94401F6091700166FB662760F970E0B7
:103F100085E00E94401F80917001082E000C990BD3
:103F2000692F661F6627661F70E086E00E94401FAB
:103F300060915F0170E08AE00E94401F4091600143
:103F400050916101609162017091630123E08BE007
:103F50000E94191F409164015091650160916601B2
:103F60007091670123E08CE00E94191F609170013D
:103F7000617070E08DE00E94401F6091700165FBF0
:103F8000662760F970E084E10E94401F6091700133
:103F900063FB662760F970E085E10E94401F609135
:103FA00070016295617070E086E10E94401F60912F
:103FB000710170E087E10E94401F409172015091B1
:103FC0007301609174017091750123E088E10E9492
:103FD000191F40917601509177016091780170919D
:103FE000790123E089E10E94191F60917A017091A3
:103FF0007B018AE10E94401F40917C0150917D012C
:1040000060917E0170917F0123E08BE10E94191F76
:10401000409168015091690160916A0170916B0152
:1040200020E08EE10E94191F40916C0150916D01BA
:1040300060916E0170916F0120E08FE10E94191F65
:10404000609170016695617070E080E20E94401F8F
:10405000D4E6F12C0BE211E083E0E82EED0ECD2F3B
:1040600082E0F81691F0E3E0FE16E9F0F1E0FF16C9
:1040700031F0F80140815181628173811AC0F801E9
:10408000448555856685778514C020E030E041E69B
:1040900055E4F801608D718D828D938D0E94BC373F
:1040A000AB01BC0106C0F80144A155A166A177A1EE
:1040B000705823E08C2F0E94191F0C5F1F4FCF5F99
:1040C000CE11CECFD65FF394DC3821F6DF91CF91BD
:1040D0001F910F91FF90EF9008958DE50E94773228
:1040E0000C94D21ECF93DF93CDB7DEB72C970FB6CB
:1040F000F894DEBF0FBECDBF8FE093E00E94C31ED9
:104100006DE071E0CE0101960E941E1DCE01019668
:104110000E94801E8AE30E94773280911F010E94D4
:104120009D1E0E946D202C960FB6F894DEBF0FBE28
:10413000CDBFDF91CF9108951F920F920FB60F92CE
:1041400011242F933F934F935F936F937F938F939C
:104150009F93AF93BF93EF93FF9380911A018130A8
:1041600049F080913C05811105C00E94F93481E03D
:104170000E94CA1CFF91EF91BF91AF919F918F91C7
:104180007F916F915F914F913F912F910F900FBE53
:104190000F901F90189593B196718091700186FDD4
:1041A00002C086E19827992349F091FB882780F97E
:1041B00092FD8260907119F08460089580E0089506
:1041C000EBE6F0E08081897E8083E8E6F0E08081A4
:1041D0008E7F8083089584B1897E84B985B186619C
:1041E00085B98091700183FF0BC080916B0086615F
:1041F00080936B00809168008160809368000895CF
:104200000C94E0200F931F93CF93C42F20E030E055
:1042100040EA51E40E94143A0E949B370E943538CC
:104220008B0101151105D9F080911B01811117C077
:10423000C11103C00E947B3306C00E948A1780917F
:104240001C0181FD0CC02FEF80E792E021508040DF
:104250009040E1F700C0000001501109E2CFCF917A
:104260001F910F910895EFE1F5E0A1E0B1E04D91CC
:104270005D916D917C911397408351836283738329
:1042800014964D915D916D917C9117974483558360
:104290006683778318968D919D910D90BC91A02D8A
:1042A00080879187A287B3870895BF92CF92DF92CC
:1042B000EF92FF920F931F93CF93DF937C01FC014A
:1042C00002A513A5D4A5C5A5818980FF18C060915A
:1042D000220170E080E090E00E9466382AE037ED2D
:1042E00043E25CE30E94143A9B01AC01B8018D2FBC
:1042F0009C2F0E94143A8B01D82FC92F2DC082FD0C
:1043000017C06091210170E080E090E00E94663863
:104310002AE037ED43E25CE30E94143A9B01AC01D2
:10432000B8018D2F9C2F0E94143A8B01D82FC92FD2
:10433000F701B6A0C7A0D0A4F1A42B2D3C2D4D2D84
:104340005F2DB8018D2F9C2F0E94D439181624F4AC
:104350000B2D1C2DDD2DCF2D20E030E040E85FE35C
:10436000B8018D2F9C2F0E94D439181624F000E03C
:1043700010E0D0E8CFE3B8018D2F9C2FDF91CF91D3
:104380001F910F91FF90EF90DF90CF90BF90089515
:104390002F923F924F925F926F927F928F929F9255
:1043A000AF92BF92CF92DF92EF92FF920F931F9343
:1043B000CF93DF93CDB7DEB7CA54D1090FB6F894C7
:1043C000DEBF0FBECDBF4B01A0901E052A2C312CA5
:1043D00022E3229DA001239D500D1124BA016250B9
:1043E0007E4F7AAF69AFFB0111922A95E9F7F4018C
:1043F0002085FB01218BF401448155816681778101
:10440000E9ADFAAD46A757A760AB71AB21FF42C03B
:104410002CE0E1E0F1E0DE01599601900D922A9541
:10442000E1F78BAB9CAB2BE231E021963FAF2EAF97
:104430002197BE016B5D7F4F7EAF6DAFCE01499678
:1044400098AF8FABFE013D96FCAFEBAF62E3A69E4B
:104450009001112427963FAF2EAF2797FEABEDAB0F
:1044600000E010E0B12C82E3829D9001839D300D2D
:104470001124C90182509E4FFC013C962396FFAF48
:10448000EEAF23979C01205F3F4F25963FAF2EAFA5
:10449000259743C02CE0EFE1F5E0BDCF2796EEADC8
:1044A000FFAD2797E00FF11FE250FE4FC082D1828F
:1044B000E282F3822396EEADFFAD23972081318116
:1044C00042815381C216D306E406F50610F4690151
:1044D0007A012396EEADFFAD2397C082D182E282AE
:1044E000F3820E946638A30192010E94BC37EDA9B5
:1044F000FEA96193719381939193FEABEDAB20E0A4
:1045000030E0A9010E94B23787FD41C0B3940C5F2F
:104510001F4F0C30110509F44CC0EBA9FCA96191A7
:10452000719181919191FCABEBAB2196EEADFFAD1A
:10453000219741905190619071902196FFAFEEAF1D
:104540002197A30192010E94143A0E94E139EDAD36
:10455000FEAD6193719381939193FEAFEDAFEFA99F
:10456000F8ADC190D190E190F190F8AFEFAB6C193C
:104570007D098E099F096B017C0197FF8FCFCC24A9
:10458000DD247601C61AD70AE80AF90A87CFBB20CC
:1045900029F0F1E0BF1621F090E803C090E201C0DD
:1045A00090E42596EEADFFAD25978081892B808321
:1045B000ADCFCD28CE28CF2809F4A3C1CE010D96CA
:1045C0000E940D1C9B01AC0182E3829D8001839DB2
:1045D000100D112402501E4FF801268F378F40A373
:1045E00051A3BE01635F7F4F83E491E028962FAF14
:1045F000289729963FAF29972A964FAF2A972B964F
:104600005FAF2B970E94B71BF801628F738F848F67
:10461000958FBE01635F7F4F87E391E00E94B71BD8
:10462000F80166A377A380A791A7F18828962FADFC
:10463000289729963FAD29972A964FAD2A972B9612
:104640005FAD2B97F0FC09C0F4016081718182811C
:104650009381F3FC0E94143AF80162A773A784A720
:1046600095A78091FD01A81611F0F1FE0DC082E31F
:10467000829DF001839DF00D1124E250FE4F128ABD
:10468000138A148A158A54C02BE235E03CAB2BAB5D
:104690008E010F5F1F4FBE01675E7F4F7AAB69AB24
:1046A000C12CD12C76010DAB1FABEBA9FCA98190DD
:1046B0009190A190B190FCABEBABEBADFCAD419018
:1046C000519061907190FCAFEBAFA3019201C501D5
:1046D000B4010E94143A9B01AC01C701B6010E94CB
:1046E000BC366B017C01A5019401C301B2010E949B
:1046F000BC36F80161937193819391938F012BAD37
:104700003CAD69A97AA92617370779F62FEE3FEF56
:104710004FE75FE3C701B6010E94D43918166CF465
:1047200082E3829DF001839DF00D1124E250FE4F43
:1047300012A213A214A215A271C02FEE3FEF4FE7F1
:104740005FEBC701B6010E94B23787FF11C082E359
:10475000829DF001839DF00D1124E250FE4F89E906
:1047600096E7A6E9BEE782A393A3A4A3B5A356C088
:104770008DA99FA90E940D1C6DA97FA983E491E0DA
:104780000E94B71B4B015C01A701960160E070E03D
:1047900080E89FE30E94BC3620E030E040E05FE329
:1047A0000E94143A0E94B33A6B017C01209160018F
:1047B000309161014091620150916301C501B401E2
:1047C0000E94143AA70196010E94143A4B015C0121
:1047D000A701960160E070E080E89FE30E94BC368C
:1047E0009B01AC01C501B4010E94BC376B017C0187
:1047F00020E030E0A9010E94B23787FF03C0C12C3E
:10480000D12C760182E3829DF001839DF00D11246D
:10481000E250FE4FC2A2D3A2E4A2F5A282E3829D9F
:104820008001839D100D112402501E4FF8018189D3
:1048300081FD69C089AD9AAD0E9455216B017C0153
:104840008090370590903805A0903905B0903A05D2
:10485000A50194010E94D43918162CF4A5019401E5
:10486000C501B40104C0A7019601C701B6010E94A9
:10487000143AF801668B778B808F918F82E3829D4B
:104880008001839D100D112402501E4FF80182A05B
:1048900093A0A4A0B5A0A501940166897789808D15
:1048A000918D0E94D43918162CF4F801868A978AC3
:1048B000A08EB18EC0923705D0923805E0923905AE
:1048C000F0923A058CE0FE013D96ABE2B5E0019036
:1048D0000D928A95E1F78CE0FE01B596AFE1B5E067
:1048E00001900D928A95E1F78091FC0180931E055D
:1048F0008F5F803109F480E08093FC010E94CC300E
:1049000002C080E001C081E0C65BDF4F0FB6F894C3
:10491000DEBF0FBECDBFDF91CF911F910F91FF90F2
:10492000EF90DF90CF90BF90AF909F908F907F904F
:104930006F905F904F903F902F9008952F923F92ED
:104940004F925F926F927F928F929F92AF92BF929F
:10495000CF92DF92EF92FF920F931F93CF93DF934B
:10496000CDB7DEB7A1970FB6F894DEBF0FBECDBFAF
:1049700090911B019111C3C18D8F3E012DE0620EFC
:10498000711C89E0D3011D928A95E9F786E08D8B31
:104990002FE4A22E21E0B22EFE0176964F0100E018
:1049A00010E0C12CD12C76013D8D232F30E03C8FBF
:1049B0002B8F902F0115110521F0013021F080E19E
:1049C00003C084E001C088E0D4018D934D01EB8DDC
:1049D000FC8D02C0F595E7959A95E2F7E0FF17C0C8
:1049E00020E030E040EC5FEBD5016D917D918D9141
:1049F0009C910E94143A1B012C019B01AC01C70140
:104A0000B6010E94D439181614F0610172010F5FCB
:104A10001F4FB4E0AB0EB11C0330110551F62090CE
:104A2000760130907701409078015090790194E0C0
:104A3000A92EBB24B39461E071E0CE0101960E94DF
:104A40001E1D80917101882E912CFE01319621E06E
:104A500031E03A8F298F890120E030E060E070E09A
:104A6000D701C601B0588E8F9F8FA8A3B9A34B8DD5
:104A70005C8D022E02C0559547950A94E2F740FFDF
:104A80002BC06F5FD8011D921D921D921C9213972F
:104A9000A401022E02C0559547950A94E2F740FF03
:104AA00003C0BB2019F007C0BB2029F0C082D1820F
:104AB000E282F38208C08E8D9F8DA8A1B9A1808368
:104AC0009183A283B38346E150E04C0F5D1F420FF8
:104AD000531FDA014C91742B2F5F3F4F34960C5FBC
:104AE0001F4F2330310519F6172F70E080E090E05A
:104AF0000E9464380E94B33A9B01AC0110932001DC
:104B0000C201B1010E94143A6D877E878F87988B0E
:104B1000B301CE0101960E94C821B4E0B0931E01FA
:104B20000E94D9280E947217BB20E9F00E94CB2076
:104B3000FE01769620E030E090E06191462F41231F
:104B400059F0AC01022E02C0559547950A94E2F740
:104B500040FF02C0609516232F5F3F4F2330310581
:104B600061F7109320010E94D92880913B0584733E
:104B700039F110913B0514FF03C086E00E94CA1C66
:104B800015FF03C087E00E94CA1CB11007C00E9435
:104B9000CB20ED8D8E2339F088E003C012FF03C0D7
:104BA00089E00E94CA1C80913C05882329F00E945C
:104BB000F9340E947B33A3C084E00E94D01C04C05F
:104BC000812F8C7109F0B0CF0E94123200917A01CE
:104BD00010917B010115110549F08FE99FE00197C4
:104BE000F1F700C0000001501109F4CF91E0B9269F
:104BF000C9F020E030E040EA50E460917C0170911F
:104C00007D0180917E0190917F010E94143A6B0199
:104C10007C0120907201309073014090740150909B
:104C2000750110C0C0907C01D0907D01E0907E01A4
:104C3000F0907F01209076013090770140907801CC
:104C400050907901AA94A110F6CEC0907101D12C98
:104C500080907C0190907D01A0907E01B0907F01BA
:104C60002401350177FA709477F870948BE2E82E7E
:104C700081E0F82E8B8D9C8D002E02C09595879536
:104C80000A94E2F780FF2AC0C601002E02C0959563
:104C900087950A94E2F7D70180FF10C094962D9172
:104CA0003D914D915C919797C501B4010E94BD362D
:104CB000F701208131814281538106C02D913D91C0
:104CC0004D915C91C301B2010E94143A0E94E139F6
:104CD000E98DFA8D60837183828393830F5F1F4F09
:104CE000298D3A8D2C5F3F4F3A8F298F34E0E30EA8
:104CF000F11C0330110509F0BDCF10921E01A196E1
:104D00000FB6F894DEBF0FBECDBFDF91CF911F91DC
:104D10000F91FF90EF90DF90CF90BF90AF909F905A
:104D20008F907F906F905F904F903F902F9008955D
:104D3000F894F999FECF92BD81BD81E08FBB80B51B
:104D40008627482F082E000C550B262F30E02423F1
:104D50003523232B39F06F3F19F060BD84E006C086
:104D600084E104C0882321F060BD84E28FBBF99AFE
:104D7000789408958091FD0190911E05981739F05F
:104D800022E3829FC001112482509E4F089580E04B
:104D900090E008958CE1EFE1F5E0DF011D928A9546
:104DA000E9F71092FD0110921E0581E08093FC014D
:104DB00010921B0608958F929F92AF92BF92CF924E
:104DC000DF92EF92FF920F931F93CF937C014A01E2
:104DD0006B01C40ED51E8B01C0E05C01A61AB70A98
:104DE000C8018A0D9B1D0C151D0599F0C11108C045
:104DF0002C2FCC0F330B232F221F2227221F01C061
:104E000021E0F80161918F01C22FC60F0E94982600
:104E1000E7CF6C2FC701880D991DCF911F910F917E
:104E2000FF90EF90DF90CF90BF90AF909F908F90CA
:104E30000C9498266AE080E090E00E94982645E570
:104E400050E06BE271E081E090E00C94DB26CF93C0
:104E5000DF9300D01F92CDB7DEB76A837B8389834F
:104E60000E94873489812DE0829FC00111244CE08B
:104E700050E06A817B819E5F0F900F900F90DF91D1
:104E8000CF910C94DB26EF92FF920F931F93CF9359
:104E9000DF93CDB7DEB72C970FB6F894DEBF0FBE09
:104EA000CDBF182F80FFD5C08AE080935B0189E1D8
:104EB00080935E0110925C0110925D0181E080930D
:104EC0005F018AE097EDA3E2BCE3809360019093D9
:104ED0006101A0936201B09363018FE692E1A3E0C8
:104EE000BBE38093640190936501A0936601B09346
:104EF000670180E090E0AAE7B4E4809368019093B2
:104F00006901A0936A01B0936B0110926C01109239
:104F10006D0110926E0110926F011092710180E08C
:104F200090E0A8ECB1E48093720190937301A09398
:104F30007401B093750180E090E0AAEFB3E4809330
:104F4000760190937701A0937801B09379012AEFCD
:104F500030E030937B0120937A0140E050E060E83C
:104F60007FE340937C0150937D0160937E017093B9
:104F70007F011092700140E050E06AE773E44093D3
:104F80002B0150932C0160932D0170932E014093BF
:104F90002F0150933001609331017093320140939F
:104FA000330150933401609335017093360180933F
:104FB000370190933801A0933901B0933A0180935F
:104FC0003B0190933C01A0933D01B0933E0180933F
:104FD0003F0190934001A0934101B093420180E0D2
:104FE00090EAACE0B7E48093430190934401A0932E
:104FF0004501B09346018093470190934801A093E7
:105000004901B0934A0180934B0190934C01A093C6
:105010004D01B0934E0180E090E0A8E4B3EC8093A2
:105020004F0190935001A0935101B093520180938E
:10503000530190935401A0935501B093560180936E
:10504000570190935801A0935901B0935A010E94BF
:105050001A2711FF10C0CE0101967C018CE0F701E8
:1050600011928A95E9F700E0B701802F0E94272767
:105070000F5F0830C9F712FF14C060E080E093E0D2
:105080000E94982660E081E093E00E94982660E00C
:1050900081E593E00E94982660E082E593E00E941B
:1050A000982613FF0AC060E08EEA93E00E949826DB
:1050B00060E08FEA93E00E9498262C960FB6F89451
:1050C000DEBF0FBECDBFDF91CF911F910F91FF903B
:1050D000EF900895F999FECF92BD81BD81E08FBB1D
:1050E00080B508958F929F92AF92BF92CF92DF9238
:1050F000EF92FF920F931F93CF934B017A016C01B4
:10510000C40ED51E8C01C0E05B01A81AB90AC50106
:10511000800F911F0C151D0599F00E946A28C1117E
:1051200008C02C2FCC0F330B232F221F2227221F26
:1051300001C021E0C22FC80FF80181938F01E7CF92
:10514000C4018E0D9F1D0E946A2821E030E0C8171F
:1051500011F020E030E0C901CF911F910F91FF9035
:10516000EF90DF90CF90BF90AF909F908F90089579
:105170001F93CF93DF93182FEB018DE0189FB001A1
:1051800011247E5F4CE050E0CE010E947228892BF2
:1051900059F48CE0FE0111928A95E9F7BE01812F46
:1051A0000E94272780E001C081E0DF91CF911F910D
:1051B00008952F923F924F925F926F927F928F92BB
:1051C0009F92AF92BF92CF92DF92EF92FF920F9396
:1051D0001F93CF93DF93CDB7DEB7EC970FB6F8945C
:1051E000DEBF0FBECDBF80911E0180FD98C790919C
:1051F000650580911C06981709F491C780911F06D8
:1052000090912006892B09F03BC310911E0112FFDB
:1052100009C080911E0522E3289FC00111248250FD
:105220009E4F02C00E94BA269093200680931F06CC
:1052300020901F06309020062114310409F46FC716
:105240000091EC05902F917000FF03C01092EC05C7
:10525000FEC08091EB058F5F853009F0982F909309
:10526000EB05E92EF12C32E13E9DF0013F9DF00D62
:105270001124EF56FA4FF0931E06E0931D06D1015C
:1052800050968C915097808B4D915D916D917C9152
:10529000DB01CA0123E0880F991FAA1FBB1F2A95B3
:1052A000D1F780839183A283B383D10114964D916A
:1052B0005D916D917C911797DB01CA0133E0880FF6
:1052C000991FAA1FBB1F3A95D1F784839583A683A4
:1052D000B783D10118964D915D916D917C911B978B
:1052E000DB01CA0143E0880F991FAA1FBB1F4A9523
:1052F000D1F780879187A287B387D1011C964D9102
:105300005D916D917C911F97DB01CA0153E0880F7D
:10531000991FAA1FBB1F5A95D1F784879587A68727
:10532000B787F10164857585868597850E94643805
:105330006093F1057093F2058093F3059093F40563
:10534000D1015E962D913D914D915C9191970E9476
:10535000BC379B01AC016093F5057093F605809313
:10536000F7059093F80560E070E080EA9FE30E9403
:10537000BC376093F9057093FA058093FB05909311
:10538000FC051092ED051092EE051092EF051092BB
:10539000F00511FD02C003FF1DC060910A06709167
:1053A0000B0680910C0690910D0660930206709397
:1053B000030680930406909305069B01AC010E94AE
:1053C000143AF101628B738B848B958B077F00936A
:1053D000EC0511C0D10152966D917D918D919C91FA
:1053E00055970E94B33A6093020670930306809328
:1053F000040690930506B2E1BE9DC001BF9D900DCD
:105400001124FC01EF56FA4F7F01118A809170013F
:1054100081FF1DC0D10151968C91519785FF17C016
:105420009A962D913D914D915C919D9760E070E031
:1054300080E89FE30E94BC376093160670931706BE
:10544000809318069093190621E0F701218B1092A2
:10545000FE051092FF051092000610920106D10180
:105460005A968D919D910D90BC91A02D89839A8320
:10547000AB83BC839C01AD0160E070E080E09FE302
:105480000E94BC374B015C01F101468C578C60A037
:1054900071A011FF4BC0F2E0F093FD05D1015296CF
:1054A000CD90DD90ED90FC905597A70196010E945C
:1054B000143A9B01AC01C301B2010E94BC364B01FE
:1054C0005C0120E030E0A9010E94B23787FF1DC0D7
:1054D00029813A814B815C81CA01B9010E94BD36A4
:1054E000A30192010E94143A9B01AC01C701B601CD
:1054F0000E94BC360E94B33A60930A0670930B0672
:1055000080930C0690930D06B8C18092FE05909290
:10551000FF05A0920006B092010610920A061092B2
:105520000B0610920C0610920D06A7C11092FD05F5
:1055300040920E0650920F0660921006709211066D
:1055400012FF0CC010920A0610920B0610920C0665
:1055500010920D06C12CD12C760124C0E091FD01E2
:10556000EF5FE03109F4E0E080911E05E81759F0A3
:10557000B2E3BE9FF0011124E250FE4FC288D388EF
:10558000E488F58803C0C12CD12C7601C701B6018F
:105590000E94B33A60930A0670930B0680930C0640
:1055A00090930D06C1010E945521698B7A8B8B8BDC
:1055B0009C8B9B01AC010E94143A69877A878B8788
:1055C0009C87D10152962D913D914D915C915597BB
:1055D0002D833E834F8358879B01AC016D817E8173
:1055E0008F8198850E94D43918160CF070C02985D7
:1055F0003A854B855C856D817E818F8198850E947F
:10560000BC369B01AC01C501B4010E94143A9B0158
:10561000AC01C301B2010E94BC3660930E067093C8
:105620000F06809310069093110620E030E0A90148
:105630000E94B23718163CF1B2E0B093FD05298103
:105640003A814B815C81CA01B9010E94BD36A30138
:1056500092010E94143A9B01AC016D817E818F8181
:1056600098850E94BC360E94B33A60930A067093F4
:105670000B0680930C0690930D068091EC058860D4
:105680008093EC05FAC0A701960169857A858B8520
:105690009C850E94BC369B01AC01C501B4010E94EF
:1056A000143A609312067093130680931406909335
:1056B000150629893A894B895C892093060630931F
:1056C0000706409308065093090633E0BBC0A701C4
:1056D00096016D817E818F8198850E94BC369B01E9
:1056E000AC01C501B4010E94143A9B01AC01C30195
:1056F000B2010E94BD3620E030E040E05FE30E944E
:10570000143A6D877E878F87988B20E030E0A9015F
:105710000E94D43918160CF098C0A30192016D852F
:105720007E858F8598890E94B23787FF8AC0A7013E
:10573000960169857A858B859C850E94BC369B0184
:10574000AC01C501B4010E94143A60931206709333
:10575000130680931406909315062D853E854F857C
:1057600058890E94B23787FF3BC089899A89AB89E3
:10577000BC898093060690930706A0930806B09311
:10578000090629853A854B855C856D817E818F81EF
:1057900098850E94B237811104C091E09093FD0575
:1057A0006CC02D813E814F81588569857A858B85B6
:1057B0009C850E94BC369B01AC01C501B4010E94CE
:1057C000143A9B01AC01C301B2010E94BC36609344
:1057D0000E0670930F0680931006909311064DC02D
:1057E0002D853E854F85588920930E0630930F06F0
:1057F000409310065093110620931206309313061F
:10580000409314065093150629813A814B815C819F
:10581000CA01B9010E94BD362D853E854F85588944
:105820000E94143AA70196010E94BD360E94B33A25
:105830006093060670930706809308069093090606
:105840001CC032E03093FD0518C010920E06109275
:105850000F06109210061092110680910A06909180
:105860000B06A0910C06B0910D068093060690934E
:105870000706A0930806B0930906186010931E014E
:1058800080919005482F50E05E8B4D8B87E0849F80
:10589000F001859FF00D1124EA59FA4F8091EB0534
:1058A0008483A0911F06B0912006BCAFABAF5E967B
:1058B000BC91BBA3EBADFCADF78DFCA3ABADBCAD18
:1058C0009096BC91BDA3EBADFCADF1A1FEA32091E0
:1058D000F9053091FA054091FB055091FC056BA14B
:1058E0007CA18B2F9F2F0E94BC366FA778AB89AB12
:1058F0009AAB20E030E0A9010E94B23787FF04C0D4
:105900001FA618AA19AA1AAA2091FD05298B309161
:1059100002063983409103064D835091040659874E
:10592000809105068D87909106069F8BA0910706B2
:10593000A88FB0910806B98FE0910906EA8FF0911F
:105940000E06FB8F20910F062C8F309110063D8F95
:10595000409111064E8F509112065FA3809113065D
:1059600088A79091140699A7A0911506AAA7B091AF
:10597000FE05BBA7E091FF05ECA7F0910006FDA78F
:10598000209101062EA730910A063BAB40910B06F1
:105990004CAB50910C065DAB80910D068EAB3BA0DD
:1059A0002CA00DA11EA18EE3C82E83ECD82E8EE272
:1059B000E82E89E3F82E412C512C3201CF8ED8A24B
:1059C000E9A2FAA23989313009F4FDC0ABADBCAD12
:1059D000313008F479C0333009F026C15A962D9140
:1059E0003D914D915C915D97C701B6010E94143ABB
:1059F0004B015C012F89388D498D5A8D69817D81DC
:105A000089859D850E94BC36A50194010E94B2370C
:105A100018168CF12B8D3C8D4D8D5E8D6BA17CA16C
:105A20008DA19EA10E94BC369B01AC010E94BD3697
:105A30006B017C012F89388D498D5A8D69817D815B
:105A400089859D850E94BD369B01AC01C701B601C9
:105A50000E94BC376B017C01BF89B983E88DED835F
:105A6000F98DF9872A8D2D873B8C2C8C0D8D1E8D01
:105A700031E0398B5AC120E030E040E05FE3C501FE
:105A8000B4010E94143A9B01AC0169817D81898532
:105A90009D850E94BC369B01AC01C701B6010E94E6
:105AA000143A9B01AC01632D722DC8010E94BC36D3
:105AB000362E272E8C01A501940169817D8189856F
:105AC0009D850E94BC367AC05A962D913D914D918C
:105AD0005C915D97C701B6010E94143A4B015C01CD
:105AE00020E030E040E05FE30E94143A9B01AC010B
:105AF00069817D8189859D850E94BD369B01AC01B0
:105B0000C701B6010E94143A9B01AC01632D722DAE
:105B1000C8010E94BC36362E272E8C012B8D3C8D61
:105B20004D8D5E8D0E94B23787FF40C02B8D3C8D1E
:105B30004D8D5E8D6BA17CA18DA19EA10E94BC3676
:105B40009B01AC010E94BD366B017C012F89388D11
:105B5000498D5A8D69817D8189859D850E94BD36DB
:105B60009B01AC01C701B6010E94BC376B017C01EF
:105B70002FA138A549A55AA56B8D7C8D8D8D9E8D45
:105B80000E94B237811103C0B2E0B98B02C0E1E0DC
:105B9000E98BFF89F983288D2D83398D39874A8DCB
:105BA0004D873B8C2C8C0D8D1E8DBFC0A5019401A3
:105BB00069817D8189859D850E94BD3669837D834C
:105BC00089879D87B2C0A70196016F89788D898DDD
:105BD0009A8D0E94143A9B01AC01632D722DC8016D
:105BE0000E94BC365B014C012FA138A549A55AA5DE
:105BF0000E94B23787FF96C02FA138A549A55AA5A4
:105C0000632D722DC8010E94BC362F89388D498DB5
:105C10005A8D0E94BC376B017C013FA028A409A5C6
:105C20001AA552E0598B81C05A962D913D914D9104
:105C30005C915D97C701B6010E94143A4B015C016B
:105C40009B01AC0169817D8189859D850E94D43944
:105C50001816D4F520E030E040E05FE3C501B40160
:105C60000E94143A9B01AC0169817D8189859D85E3
:105C70000E94BC369B01AC01C701B6010E94143AD8
:105C80009B01AC01632D722DC8010E94BC366FAB25
:105C900078AF89AF9AAF2BA53CA54DA55EA50E9414
:105CA000D43918168CF4A501940169817D81898508
:105CB0009D850E94BC3669837D8389879D873FA827
:105CC00028AC09AD1AAD31C02BA53CA54DA55EA5EC
:105CD000632D722DC8010E94BC369B01AC010E944D
:105CE000BD366B017C012BA93CA94DA95EA9698138
:105CF0007D8189859D850E94BD369B01AC01C701D0
:105D0000B6010E94BC376B017C01BBA9B983ECA929
:105D1000ED83FDA9F9872EA92D873BA42CA40DA501
:105D20001EA503C03A2C2B2C8401A7019601C301A8
:105D3000B2010E94BD362B013C012F8D38A149A133
:105D40005AA10E94B23787FF07C0A30192016F8D4D
:105D500078A189A19AA132C02FA538A949A95AA929
:105D6000632D722DC8010E94D4391816BCF03989F0
:105D70003093FD0589819D81A985BD8580930206AB
:105D800090930306A0930406B0930506E0911D06C8
:105D9000F0911E069189911129C024C02EE333ECA5
:105DA0004EE259E36F8D78A189A19AA10E94BD3678
:105DB0006F8F78A389A39AA3A30192010E94BC3696
:105DC0006B017C012BA53CA54DA55EA5632D722D15
:105DD000C8010E94D43918160CF4F4CD49894093B7
:105DE000FD05C8CF80911E0183FF3FC0ABADBCADA8
:105DF00051968C915197807349F19E96CD90DD908C
:105E0000ED90FC90D1979923D1F020911606309116
:105E1000170640911806509119066091020670917C
:105E2000030680910406909105060E94143A9B0196
:105E3000AC01C701B6010E94143A6B017C01C70195
:105E4000B6010E94A03280931A060AC01092270160
:105E5000109228011092290110922A0110921A061C
:105E600080911E01877F80931E0127E0ED89FE89C6
:105E70002E9FA0012F9F500D1124CA018A599A4FBD
:105E80009A87898780911A06A985BA8516968C9378
:105E90002091F5053091F6054091F7055091F805F0
:105EA000632D722DC8010E94143A69837A838B8313
:105EB0009C830E949B376B017C016091F10570917E
:105EC000F2058091F3059091F4050E949B374B01F8
:105ED0005C01A70196010E94BC360E9435386D8393
:105EE0007E838F8398872D813E81E985FA85318372
:105EF0002083232B41F480911E0181FF04C0816027
:105F000080931E010CC12091ED053091EE0540916A
:105F1000EF055091F005C301B2010E94BD362B017F
:105F20003C0129813A814B815C81C501B4010E9409
:105F3000BC369B01AC01C301B2010E94BC374B01CE
:105F40005C0120EC31EE44E65EE40E94143A0E94CB
:105F50009B370E943538603D57E0750781059105F4
:105F600060F427E0AD89BE892A9FF0012B9FF00DD8
:105F70001124EA59FA4F158254C0603A3FE0730782
:105F80008105910568F4A7E04D895E89A49FF00121
:105F9000A59FF00D1124EA59FA4FB1E0B5831FC057
:105FA0006034EFE17E078105910568F447E02D89B3
:105FB0003E89429FF001439FF00D1124EA59FA4FA8
:105FC00052E055830CC027E0AD89BE892A9FF001BD
:105FD0002B9FF00D1124EA59FA4F33E03583A7E0E7
:105FE0004D895E89A49FF001A59FF00D1124EA5907
:105FF000FA4F2581022E04C096958795779567956F
:106000000A94D2F74D815E8102C0440F551F2A9534
:10601000E2F7518340836115710551E085079105D1
:1060200068F427E0AD89BE892A9FF0012B9FF00D0F
:106030001124EA59FA4F7383628304C04FEF5FEF74
:106040005383428380911C06809390058F5F863036
:1060500019F080931C0602C010921C06E0911F06E6
:10606000F0912006832D922DD801868F978FA0A3C3
:10607000B1A3C092F105D092F205E092F305F0923F
:10608000F40529813A814B815C81C701B6010E94E8
:10609000BC36A50194010E94143A6093ED057093FB
:1060A000EE058093EF059093F0052091FE05309169
:1060B000FF054091000650910106632D722DC80125
:1060C0000E94B237811193C820E030E0A901632D0E
:1060D000722DC8010E94D43990911E01181614F037
:1060E00092FF04C0916090931E0119C01092200687
:1060F00010921F069091FD0180911E05891709F4E9
:1061000076C881E0890F803109F480E020911B0678
:10611000921302C080931B068093FD0168C8EC9621
:106120000FB6F894DEBF0FBECDBFDF91CF911F91A8
:106130000F91FF90EF90DF90CF90BF90AF909F9026
:106140008F907F906F905F904F903F902F90089529
:10615000CF93DF93C0911F06D09120062097C9F0FE
:106160008091EC0581608093EC056091020670914E
:10617000030680910406909105069B01AC010E94E4
:10618000143A6A8B7B8B8C8B9D8B1092200610921D
:106190001F06DF91CF9108952F923F924F925F9209
:1061A0006F927F928F929F92AF92BF92CF92DF9227
:1061B000EF92FF920F931F93CF93DF93D0911E0521
:1061C000D11101C0D0E1D150C0911B06DC1709F4F8
:1061D00016C1ED2EF12C22E3D29F80011124025032
:1061E0001E4FF801A688B788C08CD18C628D738D44
:1061F000848D958D9B01AC010E94BD36F801268DE2
:10620000378D40A151A10E94143A4B018C019B0192
:10621000AC01B501C6010E94B23787FD02C054012E
:10622000680182E38E9DF0018F9DF00D1124E250F4
:10623000FE4FC501D601828B938BA48BB58BD111F8
:1062400001C0D0E1D150DC1307C08091FD01C8131B
:1062500066C00E94A83063C022E32E9DC0012F9D1E
:10626000900D11249C0122503E4F790192E3792E2A
:10627000AD2EB12C7A9CC0017B9C900D1124FC01A9
:10628000E250FE4F6F01D11101C0D0E1D150809199
:10629000FD01D81302C00E94A8307A9C80017B9C2B
:1062A000100D112402501E4FF80186889788A08C8B
:1062B000B18CA501940162897389848995890E94B2
:1062C000B237882349F1F801628D738D848D958DE5
:1062D0009B01AC010E94BD36F801268D378D40A18F
:1062E00051A10E94143AF7012289338944895589C2
:1062F0000E94BD361B012C01A50194010E94B237FA
:10630000F80187FF05C0228A338A448A558A04C06F
:10631000828A938AA48AB58A7601DC13A9CFF2E334
:10632000CF9F8001112402501E4FCF5FC03109F46E
:10633000C0E020901E05D0911B0682E3382EC215C6
:1063400009F45BC0CC2ED12C3C9CC0013D9C900D2F
:1063500011249C0122503E4F7901F8014288538854
:1063600064887588F90182889388A488B588A50116
:106370009401C301B2010E94B23787FF24C0F80123
:10638000628D738D848D958D9B01AC010E94BD360D
:10639000F801268D378D40A151A10E94143A9B012E
:1063A000AC01C301B2010E94BD362B013C01A50125
:1063B00094010E94B23787FF06C0F701428A538AD0
:1063C000648A758ADC2F3C9CF0013D9CF00D112401
:1063D000E250FE4F26893789408D518D628973893D
:1063E000848995890E94B237811101C0DC2FCF5F6B
:1063F000C03109F4C0E08701A2CFD0931B06DF9122
:10640000CF911F910F91FF90EF90DF90CF90BF90B1
:10641000AF909F908F907F906F905F904F903F9044
:106420002F900895CF93DF930E94F41480E3EBEE56
:10643000F5E0DF011D928A95E9F7C2E4D5E083E239
:10644000FE0111928A95E9F71092200610921F061C
:10645000109265051092900581E080931C061092C1
:1064600041050E94C414809140058F878BB1837EC3
:1064700090913F05892B8BB98BB18F71909140051D
:10648000892B8BB9DF91CF9108950E94BA26892B71
:1064900019F082E00C94DA1C08951F920F920FB647
:1064A0000F9211248F939F93EF93FF938091100786
:1064B000E82FF0E0E955F94F90819093C6008F5F87
:1064C000893609F480E0809310079091A60689131D
:1064D00005C08091C1008F7D8093C100FF91EF9135
:1064E0009F918F910F900FBE0F901F901895E09184
:1064F000A60691E09E0F993631F490E004C02091F9
:106500003B0524FD0FC0209110079217C1F3F0E066
:10651000E955F94F80839093A6068091C10080626F
:106520008093C100089590911B01911108C08111C1
:1065300002C0439802C086FD439A10922501089537
:106540004F925F926F927F928F929F92AF92BF9283
:10655000CF92DF92EF92FF92CF936B017C01C091BB
:10656000230180906C0190906D01A0906E01B0901D
:106570006F01409068015090690160906A017090CD
:106580006B01A3019201C501B4010E94D43987FFB8
:106590001AC06C2F70E080E090E00E9466382AE01C
:1065A00037ED43E25CE30E94143A9B01AC01C70162
:1065B000B6010E94143A6B017C01A30192010E9472
:1065C000D43987FD0AC04092270150922801609279
:1065D000290170922A018FEF47C0A5019401C701DC
:1065E000B6010E94B2371816E4F020E030E0A901AD
:1065F000C701B6010E94B237811109C0109227016C
:10660000109228011092290110922A012DC0809227
:10661000270190922801A0922901B0922A0181E0DD
:1066200023C0C0922701D0922801E0922901F09264
:106630002A01A5019401C701B6010E94BC36209130
:10664000A2063091A3064091A4065091A5060E948F
:10665000143A0E94A13820E030E040E85FE30E9455
:10666000BD360E943538862FCF91FF90EF90DF9096
:10667000CF90BF90AF909F908F907F906F905F90E2
:106680004F9008958093B300811104C08091B000B1
:106690008F7703C08091B00080688093B000089528
:1066A00090911B01911126C081110EC010922701FB
:1066B000109228011092290110922A018091B000B5
:1066C0008F778093B00014C0803111F42D9801C0F1
:1066D0002D9A9091700191FF05C0803219F440E02D
:1066E00050E0BA01CB01BA010E94A0320E944233AD
:1066F000109225010895CF92DF92EF92FF921F939F
:10670000CF93DF930E948A1780911C01882309F49C
:10671000F6C00E94BA26009771F4C091880180915A
:106720008901C82BC0908B01D0908C01E0908D0125
:10673000F0908E0106C0FC01C189C6A4D7A4E0A8D0
:10674000F1A88091700181FF03C080E20E94B81C13
:10675000DC2FD07311E0C07490911C01992309F4CF
:10676000CEC080911B018111CAC090FFC5C080912D
:106770001A01282F207C09F474C092FD12C01092D7
:10678000240140E050E0BA0180E00E94503380E0F4
:106790000E94933290911C019D7F946090931C0104
:1067A000ABC08038E1F483EA92E00E94C31E8CE023
:1067B00092E00E94C31E0E946D2040E050E0BA01AA
:1067C00080E00E94503380E00E9493320E94F414D3
:1067D00080911B01811193C00E948A17F9CF8034E8
:1067E00019F49F7D90931C0180911C0183FF84C04C
:1067F000909189019923C1F081FD16C080917001AB
:1068000081FF06C080911E01886080931E010CC02C
:10681000B701A6018D2F0E94503341E060E070E087
:1068200080E890E40E94022180918801882371F021
:1068300080911C0181FD0AC08C2F0E94933241E09F
:1068400060E070E080E89FE30E94022190911C01CB
:1068500091FD52C0906190931C0182E00E94DA1C6D
:106860004BC0909124019923C9F191FF0DC08091F3
:1068700089018823B1F040E050E0BA0180E00E9435
:1068800050331093240138C09C70B1F1809189017C
:1068900081110AC08091240183FF03C082E00E941D
:1068A000DA1C1092240128C083EA92E00E94C31EE1
:1068B00085E192E00E94C31E0E946D2080917001CC
:1068C00081FF06C080911E01886080931E01E2CF87
:1068D000B701A6018D2F0E945033DCCF80911E019D
:1068E00083FF0AC0B701A6018D2F0E94503380910B
:1068F0001E01877F80931E010E948A172DCFDF9192
:10690000CF911F91FF90EF90DF90CF9008950E945C
:1069100045320E947B3380911B01811108C00E9487
:10692000BA26892BB1F780911A01883091F3089526
:10693000CF93DF9300D000D01F92CDB7DEB79091F8
:106940001A019230A9F04A835B836C837D8389832B
:106950000E9487344A815B816C817D8189810F909F
:106960000F900F900F900F90DF91CF910C945033B8
:106970000F900F900F900F900F90DF91CF9108958F
:10698000CF93DF93239AC0EBD0E083E0888384E049
:106990008093B100259A20916C0130916D01409156
:1069A0006E0150916F016091680170916901809151
:1069B0006A0190916B010E94BC369B01AC0160E0C2
:1069C00070E08EE793E40E94BC376093A206709358
:1069D000A3068093A4069093A50688818F77888369
:1069E000DF91CF91089561E071E088E991E00C9426
:1069F0001E1D80913B0584FD1FC080E10E94DA1CB2
:106A00008091B0008F778093B000439890911A01E5
:106A1000892F8C7221F480911E01867069F0943068
:106A200031F480913C05811105C086E001C083E00E
:106A30000E94CA1C0C94F41408951F920F920FB672
:106A40000F9211242F933F934F935F936F937F93F4
:106A50008F939F93AF93BF93EF93FF93E091C60003
:106A6000E13271F028F4E83179F40E94F93456C02B
:106A7000EF3321F0EE3741F482E003C081E001C042
:106A800088E00E94DA1C4AC0E7FF37C08E2F90E0F2
:106A9000FC01E458F109ED31F10508F03FC0E65979
:106AA000FF4F0C945F3B80E2ECCF80911A0185FF91
:106AB00035C080E4E6CF81E00DC082E00BC084E009
:106AC00009C088E007C080E105C080E203C080E41F
:106AD00001C080E80E94C11C21C081E00BC082E09F
:106AE00009C084E007C088E005C080E103C080E2FF
:106AF00001C080E40E94B81C11C0A091FA0181E09D
:106B00008A0F813809F480E09091FB01891731F0F8
:106B1000B0E0AF5DB94FEC938093FA01FF91EF9134
:106B2000BF91AF919F918F917F916F915F914F91A5
:106B30003F912F910F900FBE0F901F901895EF92DD
:106B4000FF920F931F93CF93DF931F92CDB7DEB7C2
:106B50008C017B018091700185FF26C020911A0174
:106B6000203211F1C80129830E94E31C2981882366
:106B7000D9F081E080931D01283041F00E94F93462
:106B800082E00E94CA1C0E947B330EC088E00E94F3
:106B9000DA1C0E947B3380911B01811105C080911A
:106BA0001A018111F6CFEACF80911A01823059F192
:106BB0000E947B3380911B01811125C09091FD01C2
:106BC0008091FC01981303C00E944532F1CFB701B8
:106BD000C8010E94C821811116C08091700181FFF7
:106BE00012C0F701808584FF0EC044815581668103
:106BF000778180E10F90DF91CF911F910F91FF90EE
:106C0000EF900C9498340F90DF91CF911F910F91DA
:106C1000FF90EF9008958F929F92AF92BF92CF9284
:106C2000DF92EF92FF920F931F93CF93DF937C013C
:106C30006B01DC01EC91F0E0EF5EF84F9081EF0129
:106C40009D3221F42296918101E007C09B3211F020
:106C5000219602C02296918100E0912CF0E010E094
:106C600020E030E0A9015E01E0EDE90FEA30D0F468
:106C7000FF5FF93098F491101150A5E0B0E00E9448
:106C8000653BDC01CB01880F991FAA1FBB1F9C012C
:106C9000AD012E0F311D411D511D0AC0911008C0BC
:106CA0001F5F06C0EE3F41F4911006C099249394F3
:106CB0002196D5019C91D7CFFF2309F44FC0CA017B
:106CC000B9010E9464384B015C0120E030E0A90169
:106CD0000E94B237882349F11F3F64F42AE037ED60
:106CE00043E25CE3C501B4010E94143A4B015C012C
:106CF0001E5FF2CF1F3F59F42DEC3CEC4CEC5DE3F2
:106D0000C501B4010E94143A4B015C010EC011236D
:106D100061F020E030E040E251E4C501B4010E949E
:106D2000143A4B015C011150F2CF002351F0B7FA35
:106D3000B094B7F8B094F60180829182A282B382B7
:106D400006C0D6018D929D92AD92BC921397C1510F
:106D5000D740C150F701C08381E001C080E0DF91DE
:106D6000CF911F910F91FF90EF90DF90CF90BF9048
:106D7000AF909F908F9008955058BB27AA270E94EC
:106D8000D4360C946E390E94353938F00E943C3963
:106D900020F039F49F3F19F426F40C940B390EF4CB
:106DA000E095E7FB0C94DC38E92F0E94933958F307
:106DB000BA17620773078407950720F079F4A6F5E0
:106DC0000C94CD390EF4E0950B2EBA2FA02D0B01AB
:106DD000B90190010C01CA01A0011124FF27591B20
:106DE00099F0593F50F4503E68F11A16F040A22F26
:106DF000232F342F4427585FF3CF46953795279597
:106E0000A795F0405395C9F77EF41F16BA0B620B95
:106E1000730B840BBAF09150A1F0FF0FBB1F661FDC
:106E2000771F881FC2F70EC0BA0F621F731F841F1F
:106E300048F4879577956795B795F7959E3F08F045
:106E4000B0CF9395880F08F09927EE0F9795879507
:106E500008950E94353960F080E891E009F49EEFD2
:106E60000E943C3928F040E851E071F45EEF0CC01C
:106E70000C940B390C94CD39E92FE0780E949339AA
:106E800040F3092E052AB1F326173707480759079B
:106E900038F00E2E07F8E02569F0E025E0640AC01E
:106EA000EF6307F8009407FADB01B9019D01DC01EB
:106EB000CA01AD01EF930E94D3370E946E390E9440
:106EC0006C375F91552339F02BED3FE049E450FDDD
:106ED00049EC0C94BD360895DF93DD27B92FBF77B9
:106EE00040E85FE31616170648075B0718F4D92F2A
:106EF0000E94D9399F938F937F936F930E94F33AA7
:106F0000EEE0F1E00E940E390E946E392F913F9120
:106F10004F915F910E94273ADD2351F09058A2EAE9
:106F20002AED3FE049EC5FE3D0785D270E94D4363C
:106F3000DF910C946E390E94B53990F09F3748F478
:106F4000911116F40C94CE3960E070E080E89FE374
:106F5000089526F01B16611D711D811D0C94E238E9
:106F60000C94FD380E94B83808F481E008950E941E
:106F70004539E3950C947F390E94D0370C946E39D3
:106F80000E943C3958F00E94353940F029F45F3FA7
:106F900029F00C94DC3851110C94CE390C940B3937
:106FA0000E94933968F39923B1F3552391F3951B0C
:106FB000550BBB27AA2762177307840738F09F5F1A
:106FC0005F4F220F331F441FAA1FA9F335D00E2E87
:106FD0003AF0E0E832D091505040E695001CCAF7F4
:106FE0002BD0FE2F29D0660F771F881FBB1F2617B7
:106FF00037074807AB07B0E809F0BB0B802DBF018E
:10700000FF2793585F4F3AF09E3F510578F00C945C
:10701000DC380C94CE395F3FE4F3983ED4F3869588
:1070200077956795B795F7959F5FC9F7880F911D7D
:107030009695879597F90895E1E0660F771F881F69
:10704000BB1F621773078407BA0720F0621B730B1C
:10705000840BBA0BEE1F88F7E09508950E9435382F
:107060006894B1110C94CE3908950E949B3988F030
:107070009F5798F0B92F9927B751B0F0E1F0660FFC
:10708000771F881F991F1AF0BA95C9F714C0B1303D
:1070900091F00E94CD39B1E008950C94CD39672F5D
:1070A000782F8827B85F39F0B93FCCF3869577956C
:1070B0006795B395D9F73EF4909580957095619555
:1070C0007F4F8F4F9F4F0895E89409C097FB3EF480
:1070D00090958095709561957F4F8F4F9F4F992325
:1070E000A9F0F92F96E9BB279395F69587957795A3
:1070F0006795B795F111F8CFFAF4BB0F11F460FF63
:107100001BC06F5F7F4F8F4F9F4F16C0882311F0BA
:1071100096E911C0772321F09EE8872F762F05C0CE
:10712000662371F096E8862F70E060E02AF09A9569
:10713000660F771F881FDAF7880F9695879597F95E
:1071400008950E94B53990F09F3748F4911116F0D8
:107150000C94CE3960E070E080E89FEB089526F44F
:107160001B16611D711D811D0C94E2380C94FD38B5
:10717000990F0008550FAA0BE0E8FEEF1616170648
:10718000E807F907C0F012161306E407F50798F0B0
:10719000621B730B840B950B39F40A2661F0232BC9
:1071A000242B252B21F408950A2609F4A140A69545
:1071B0008FEF811D811D089597F99F6780E870E02A
:1071C00060E00895882371F4772321F09850872B8D
:1071D000762F07C0662311F499270DC09051862B96
:1071E00070E060E02AF09A95660F771F881FDAF743
:1071F000880F9695879597F908959F3F31F09150A4
:1072000020F4879577956795B795880F911D96958A
:10721000879597F908959FEF80EC0895DF93CF93BA
:107220001F930F93FF92EF92DF927B018C01689482
:1072300006C0DA2EEF010E94273AFE01E894A591DC
:107240002591359145915591A6F3EF010E94D436D1
:10725000FE019701A801DA9469F7DF90EF90FF90A3
:107260000F911F91CF91DF91089500240A94161673
:10727000170618060906089500240A941216130624
:107280001406050608950C940B390E949B39D8F317
:10729000E894E0E0BB279F57F0F02AED3FE049EC8F
:1072A00006C0EE0FBB0F661F771F881F28F0B23A8B
:1072B00062077307840728F0B25A620B730B840BC2
:1072C000E3959A9572F7803830F49A95BB0F661F54
:1072D000771F881FD2F790480C94FF38092E03942B
:1072E000000C11F4882352F0BB0F40F4BF2B11F4B3
:1072F00060FF04C06F5F7F4F8F4F9F4F0895EF93E4
:10730000E0FF07C0A2EA2AED3FE049EC5FEB0E94F4
:10731000D4360E946E390F90039401FC9058EBE331
:10732000F1E00C94093B57FD9058440F551F59F05C
:107330005F3F71F04795880F97FB991F61F09F3F62
:1073400079F087950895121613061406551FF2CF8B
:107350004695F1DF08C0161617061806991FF1CFDB
:10736000869571056105089408950E949B39A0F0E7
:10737000BEE7B91788F4BB279F3860F41616B11D15
:10738000672F782F8827985FF7CF86957795679531
:10739000B11D93959639C8F30895E894BB276627E5
:1073A0007727CB0197F908950E94B83808F48FEF3A
:1073B00008959B01AC0160E070E080E89FE30C94CD
:1073C000BC370E949B3958F19E5760F19851A0F04C
:1073D000E9F0983020F5092E9927660F771F881F4E
:1073E000991F0A94D1F712C0062E672F782F88278D
:1073F000985F11F4000C07C0993FB4F38695779518
:1074000067959395D9F7611D711D811D3EF4909587
:107410008095709561957F4F8F4F9F4F0895689429
:107420000C94CE390C94CD390E94273A0C946E39C5
:107430000E94353938F00E943C3920F0952311F034
:107440000C94DC380C940B3911240C94CE390E9426
:10745000933970F3959FC1F3950F50E0551F629FCC
:10746000F001729FBB27F00DB11D639FAA27F00D9D
:10747000B11DAA1F649F6627B00DA11D661F829FC4
:107480002227B00DA11D621F739FB00DA11D621FA9
:10749000839FA00D611D221F749F3327A00D611DC6
:1074A000231F849F600D211D822F762F6A2F1124A8
:1074B0009F5750409AF0F1F088234AF0EE0FFF1FDB
:1074C000BB1F661F771F881F91505040A9F79E3F32
:1074D000510580F00C94DC380C94CE395F3FE4F316
:1074E000983ED4F3869577956795B795F795E79588
:1074F0009F5FC1F7FE2B880F911D9695879597F991
:1075000008950E949B39E8F09E37E8F09639B8F468
:107510009E3848F4672F782F8827985FF9CF869593
:107520007795679593959539D0F3B62FB1706B0F1A
:10753000711D811D20F487957795679593950C941F
:10754000E2380C94FD380C94CE399F930E94453953
:107550000F9007FCEE5F0C947F3919F416F40C942D
:107560000B390C94FD380E949B39B8F39923C9F369
:10757000B6F39F57550B87FF0E94023B0024A0E6FD
:1075800040EA900180585695979528F4805C660FE4
:10759000771F881F20F026173707480730F4621B33
:1075A000730B840B202931294A2BA6951794079435
:1075B000202531254A2758F7660F771F881F20F0AE
:1075C00026173707480730F4620B730B840B200D26
:1075D000311D411DA09581F7B901842F9158880F65
:1075E0009695879508959B01AC010C94143A0E94DE
:1075F000B53930F09F3710F40C94CE390C94E23842
:107600000C94FD3891505040660F771F881FD2F7B9
:1076100008959F938F937F936F93FF93EF939B01B5
:10762000AC010E94143AEF91FF910E940E392F9104
:107630003F914F915F910C94143A991B79E004C0EB
:10764000991F961708F0961B881F7A95C9F78095A1
:107650000895AA1BBB1B51E107C0AA1FBB1FA61799
:10766000B70710F0A61BB70B881F991F5A95A9F7EB
:1076700080959095BC01CD010895A1E21A2EAA1B18
:10768000BB1BFD010DC0AA1FBB1FEE1FFF1FA217D2
:10769000B307E407F50720F0A21BB30BE40BF50BCF
:1076A000661F771F881F991F1A9469F76095709558
:1076B000809590959B01AC01BD01CF010895EE0F1F
:1076C000FF1F0590F491E02D09940E94703BA59F47
:1076D000900DB49F900DA49F800D911D11240895CD
:1076E000A29FB001B39FC001A39F700D811D112403
:1076F000911DB29F700D811D1124911D0895FB01F4
:10770000DC0104C08D910190801921F4415050405A
:0C771000C8F7881B990B0895F894FFCF70
:00000001FF
